:020000040000FA
:100000002EEF35F0F76A140FF66E000EF722090096
:10001000F5501200000000000000005F0000000723
:10002000000700147F147F14242A7F2A1223130848
:10003000646236495522500005030000001C22412D
:10004000000041221C0014083E081408083E08085D
:100050000050300000080808080800606000002018
:10006000100804023E5149453E00427F4000426173
:100070005149462141454B311814127F10274545FF
:1000800045393C4A49493001710905033649494916
:1000900036064949291E0036360000005636000053
:1000A00008142241001414141414004122140802EC
:1000B00001510906324979413E7E1111117E7F4975
:1000C0004949363E414141227F4141221C7F4949F5
:1000D00049417F090909013E4149497A7F080808D9
:1000E0007F00417F41002040413F017F08142241B1
:1000F0007F404040407F020C027F7F0408107F3E1B
:100100004141413EF76A140FF66E010EF7220900D5
:10011000F55012007F090909063E4151215E7F0911
:10012000192946464949493101017F01013F4040B3
:10013000403F1F2040201F3F4038403F63140814B9
:100140006307087008076151494543007F4141003A
:1001500002040810200041417F0004020102044013
:1001600040404040000102040020545454787F482D
:100170004444383844444420384444487F38545434
:100180005418087E0901020C5252523E7F080404A2
:100190007800447D40002040443D007F102844000A
:1001A00000417F40007C041804787C0804047838FF
:1001B000444444387C14141408081414187C7C0833
:1001C0000404084854545420043F4440203C404018
:1001D000207C1C2040201C3C4030403C44281028FF
:1001E000440C5050503C4464544C44000836410088
:1001F00000007F0000004136080010080810087851
:1002000046414678F76A140FF66E020EF72209008F
:10021000F55012004272696768746E65737300006E
:10022000F76A300FF66E020EF7220900F550120041
:1002300041646A7573740000F76A480FF66E020E27
:10024000F7220900F550120054656368446573692C
:10025000676E2E626500F76A660FF66E020EF72271
:100260000900F5501200566F703D202575200000E2
:10027000F76A800FF66E020EF7220900F5501200A1
:100280000000F76A920FF66E020EF7220900F55091
:10029000120020496E7365727420436172642020DD
:1002A0000000F76AB20FF66E020EF7220900F55051
:1002B0001200737461743D20254C78200000F76AA9
:1002C000CE0FF66E020EF7220900F55012006163A0
:1002D0006D6434313D2025782000F76AEA0FF66E10
:1002E000020EF7220900F55012002020534420424C
:1002F0006F6F74696E6720200000F76A0A0FF66E50
:10030000030EF7220900F55012004D4D43204D4FCA
:1003100044452000F76A240FF66E030EF722090009
:10032000F5501200204D4D4320426F6F74696E6787
:1003300020200000F76A440FF66E030EF722090032
:10034000F550120053656356423D256C78200A0D26
:100350000000F76A620FF66E030EF7220900F550EF
:10036000120042705365633D20256C78200A0D0011
:10037000F76A800FF66E030EF7220900F55012009F
:100380002121204270536563206973206E6F7420B1
:10039000353132202121200A0D00F76AAA0FF66EAE
:1003A000030EF7220900F550120053656370436C89
:1003B000753D202578200A0D0000F76ACA0FF66EF9
:1003C000030EF7220900F5501200525365633D20D9
:1003D000254C78200A0D0000F76AE80FF66E030E30
:1003E000F7220900F55012004661744E3D20257831
:1003F000200A0D00F76A040FF66E040EF7220900BA
:10040000F5501200536563466174313D20254C78E8
:10041000200A0D00F76A240FF66E040EF722090079
:10042000F5501200464154315F6C62615F73746134
:1004300072743D20254C78200A0D0000F76A4C0F9D
:10044000F66E040EF7220900F55012005370466153
:10045000743D20254C78200A0D00F76A6A0FF66E6D
:10046000040EF7220900F550120052446972456EDD
:10047000744E3D20254C78200A0D0000F76A8C0F41
:10048000F66E040EF7220900F55012005365635210
:100490006F6F744469723D256C78200A0D00F76A0D
:1004A000AE0FF66E040EF7220900F5501200456EED
:1004B00064536563526F6F744469723D256C782094
:1004C0000A0D0000F76AD40FF66E040EF722090039
:1004D000F55012005365637046415433323D256C2C
:1004E00078200A0D0000F76AF60FF66E040EF72268
:1004F0000900F5501200436C75526F6F74446972B5
:100500005F46415433323D256C78200A0D00F76A6E
:100510001E0FF66E050EF7220900F55012006C62F0
:1005200061526F6F744469723D256C78200A0D002A
:10053000F76A400FF66E050EF7220900F55012001B
:100540005363616E6E696E670000F76A5A0FF66E4C
:10055000050EF7220900F55012002A2A736563730D
:1005600063616E3D256C75200000F76A7A0FF66EA8
:10057000050EF7220900F5501200726F7773636160
:100580006E3D256C75200000F76A980FF66E050E1B
:10059000F7220900F5501200726F777363616E31B4
:1005A0003D256C752000F76AB60FF66E050EF72232
:1005B0000900F5501200726F777363616E323D254A
:1005C0006C750A0D0000F76AD60FF66E050EF7225D
:1005D0000900F550120044454C200000F76AEC0F6A
:1005E000F66E050EF7220900F55012004C464E201B
:1005F0000000F76A020FF66E060EF7220900F550AA
:100600001200454E44312000F76A180FF66E060EB0
:10061000F7220900F5501200454E44322000F76AD7
:100620002E0FF66E060EF7220900F5501200202854
:10063000726F6F74292025750000F76A4A0FF66EF5
:10064000060EF7220900F550120046494C453D20A0
:100650000000F76A620FF66E060EF7220900F550E9
:1006600012006469725F6E756D6265723D2575205A
:100670000000F76A820FF66E060EF7220900F550A9
:10068000120063757272656E74436C757374657273
:100690003D25386C75200A0D0000F76AAA0FF66E2A
:1006A000060EF7220900F55012006E657874436C4F
:1006B00075737465723D25386C75200A0D00F76AF4
:1006C000CE0FF66E060EF7220900F55012005449BF
:1006D00054320000F76AE40FF66E060EF7220900A6
:1006E000F5501200545045310000F76AFA0FF66ECB
:1006F000060EF7220900F550120054434F4E000039
:10070000F76A100FF66E070EF7220900F550120077
:100710005452434B0000F76A260FF66E070EF7227D
:100720000900F550120054414C420000F76A3C0F9A
:10073000F66E070EF7220900F550120054454E439D
:100740000000F76A520FF66E070EF7220900F55007
:100750001200545945520000F76A680FF66E070EF2
:10076000F7220900F5501200434F4D4D0000F76A83
:100770007E0FF66E070EF7220900F55012002020BA
:100780002020202020202020202020202020202069
:10079000202020202020202020200000F76AAC0FFD
:1007A000F66E070EF7220900F55012006B627073A7
:1007B0003D202575200A0D00F76AC80FF66E070E5A
:1007C000F7220900F55012006B6270735F64656375
:1007D0003D20256C75200A0D0000F76AEA0FF66EC1
:1007E000070EF7220900F550120020736563735F4E
:1007F000746F743D256C75200000F76A0A0FF66E61
:10080000080EF7220900F55012007461675F7369E2
:100810007A653D20256C75200A0D0000F76A2C0FC3
:10082000F66E080EF7220900F55012002D20536FC6
:100830006E67205469746C65202D0000F76A4C0FB8
:10084000F66E080EF7220900F55012002D2D20201B
:1008500041727469737420202D2D0000F76A6C0FAB
:10086000F66E080EF7220900F5501200205642528B
:100870002000F76A820FF66E080EF7220900F55085
:1008800012000A0D303230202D204563686F4D7004
:1008900033204D4D432F5344206D703320506C61F5
:1008A000796572200A0D0A0D0000F76ABA0FF66E1C
:1008B000080EF7220900F5501200204563686F4DBD
:1008C00070332076312E34200000F76ADA0FF66E8E
:1008D000080EF7220900F55012004D4D432F5344E6
:1008E000204361726400F76AF60FF66E080EF72275
:1008F0000900F550120020204D703320506C6179B2
:10090000657220200000F76A160FF66E090EF722B6
:100910000900F5501200446961677300F76A2C0FF3
:10092000F66E090EF7220900F5501200536875663D
:10093000666C6500F76A440FF66E090EF72209002F
:10094000F55012004D4D432F534420696E697420B9
:10095000646F6E65200A0D00F76A680FF66E090E67
:10096000F7220900F55012004D4D432F53442072D9
:1009700065616420626F6F7420646F6E650A0D207C
:100980000000F76A920FF66E090EF7220900F55083
:100990001200767320696E697420646F6E650A0DAB
:1009A0002000F76AB20FF66E090EF7220900F55023
:1009B0001200546F74616C20536F6E67733D202575
:1009C0004C75200A0D00F76AD60FF66E090EF72255
:1009D0000900F55012006469725F6E756D62657290
:1009E0002025753D2000F76AF60FF66E090EF722F6
:1009F0000900F5501200746F74616C646972733D84
:100A0000202575200A0D0000F76A180FF66E0A0EF1
:100A1000F7220900F550120063757272656E7473E7
:100A20006F6E673D25334C752F254C752000F76A96
:100A30003E0FF66E0A0EF7220900F55012006C62A6
:100A4000615F73746172743D256C75200000F76AF4
:100A50005E0FF66E0A0EF7220900F5501200736F52
:100A60006E675F6C62615F6C656E6774683D256C74
:100A700075200A0D0000F76A860FF66E0A0EF7223F
:100A80000900F5501200737461727420706C617902
:100A9000696E672E2E0A0D00F76AA80FF66E0A0E11
:100AA000F7220900F5501200204469726563746FE3
:100AB0007269657320200000F76AC80FF66E0A0E8F
:100AC000F7220900F55012002063757272656E748A
:100AD0006469723D202575200A0D0000F2CF98F35D
:100AE000F29E010EA96EA69CA69EA680A8500301A8
:100AF00098BFF28E010B016EE8B003D00101CE95D4
:100B000002D00101CE85F2CF98F3F29E020EA96EBB
:100B1000A69CA69EA680A850030198BFF28E010B4A
:100B2000016EE8B003D00101CE9702D00101CE875B
:100B300080AA2FD0CEA517D0010EA96EA86AA69CB8
:100B4000A69EA684F2CF00F0F29E0F01550EA76E6E
:100B5000AA0EA76EA682A6B2FED7A6940050F212E5
:100B60000101CE9516D0010EA96EA86EA69CA69E78
:100B7000A684F2CF00F0F29E0F01550EA76EAA0ECA
:100B8000A76EA682A6B2FED7A6940050F21201016B
:100B9000CE8584A030D0CEA717D0020EA96EA86A49
:100BA000A69CA69EA684F2CF00F0F29E0F01550EE1
:100BB000A76EAA0EA76EA682A6B2FED7A694005074
:100BC000F2120101CE9717D0020EA96E010EA86E87
:100BD000A69CA69EA684F2CF00F0F29E0F01550EB1
:100BE000A76EAA0EA76EA682A6B2FED7A694005044
:100BF000F2120101CE870001D2EF36F0F2CF98F366
:100C0000F29EA96AA69CA69EA680A850030198BF42
:100C1000F28E0201B56FB5517F0816E3A00EB56FD5
:100C2000A96AA86EA69CA69EA684F2CF00F0F29EAA
:100C30000F01550EA76EAA0EA76EA682A6B2FED70A
:100C4000A6940050F21202010001D4EF36F0030E18
:100C5000EA6E9E0EE96EEF500DE0060E016E006A20
:100C6000002EFED7012EFBD77B0E006E002EFED786
:100C7000EF2EF3D7000C080E0501CA6FCA530CE023
:100C8000839AC951800B02E1839801D08388838ABB
:100C9000D890C937CA07F2D70001000C8392839617
:100CA000C7C5C9F5E8DF8386000C0501C551070BF0
:100CB0004009C66FC76F0001F1DF0501C4517F0B0A
:100CC0008009C66FC76F0001E9DF000C838283963D
:100CD000C8C5C9F5D0DF8386000C0501C46BC56BA0
:100CE0000001E3DF010E0201BA6FF80EB96FB953CC
:100CF00002E1BA530AE00501C86B0001E7DF020117
:100D0000B951D8B4BA07B907F2D70001A9EF06F074
:100D10008382838683940A0E03019E6F000197DF0E
:100D20008384210E0501C76F0001B8DFB5C2C7F586
:100D3000B5DF130E0501C76F0001B0DF200E0501FE
:100D4000C76F0001ABDF090E0501C76F0001A6DF09
:100D5000C4D7080E0501C76F0001A0DF0C0E050106
:100D6000C76F00019BDF000C0201B851C70803E107
:100D7000800EB86FE2D0B851FC0803E1810EB86F65
:100D8000DCD0B851E90803E1820EB86FD6D0B85173
:100D9000E20803E1830EB86FD0D0B851E40803E154
:100DA000840EB86FCAD0B851E00803E1850EB86F61
:100DB000C4D0B851E50803E1860EB86FBED0B85173
:100DC000E70803E1870EB86FB8D0B851EA0803E12D
:100DD000880EB86FB2D0B851EB0803E1890EB86F36
:100DE000ACD0B851E80803E18A0EB86FA6D0B8516C
:100DF000EF0803E18B0EB86FA0D0B851EE0803E105
:100E00008C0EB86F9AD0B851EC0803E18D0EB86F14
:100E100094D0B851C40803E18E0EB86F8ED0B8518B
:100E2000C50803E18F0EB86F88D0B851C90803E137
:100E3000900EB86F82D0B851E60803E1910EB86FFA
:100E40007CD0B851C60803E1920EB86F76D0B85185
:100E5000F40803E1930EB86F70D0B851F60803E1BF
:100E6000940EB86F6AD0B851F20803E1950EB86FCE
:100E700064D0B851FB0803E1960EB86F5ED0B8514C
:100E8000F90803E1970EB86F58D0B83D03D0980E1B
:100E9000B86F53D0B851D60803E1990EB86F4DD052
:100EA000B851DC0803E19A0EB86F47D0B851F80882
:100EB00003E19B0EB86F41D0B851A30803E19C0E2B
:100EC000B86F3BD0B851D80803E19D0EB86F35D04C
:100ED000B851D70803E19E0EB86F2FD0B8518308E0
:100EE00003E19F0EB86F29D0B851E10803E1A00ECD
:100EF000B86F23D0B851ED0803E1A10EB86F1DD033
:100F0000B851F30803E1A20EB86F17D0B851FA0830
:100F100003E1A30EB86F11D0B851F10803E1A40E9C
:100F2000B86F0BD0B851D10803E1A50EB86F05D04A
:100F3000B851DF0802E1A60EB86F0001C5EF07F057
:100F400083828396080E0501C96FC95310E0839A06
:100F5000030E006E002EFED7C851010B02E18398EC
:100F600001D08388838AD890C833C907EED7838697
:100F70000001000C0201B8511F0802E38BD006D01B
:100F8000B8517F0803E20001EFD60201B8511F08F3
:100F900001E380D0B851A60801E27CD0B66BB6510F
:100FA00004086AE3B8514F081EE3B851E00F050D7D
:100FB000F350D06BCF6FB651CF250501C86F000E2F
:100FC0000201D0210501C96F036EC851F2CFCAF5E5
:100FD000F29E000102EC00F00501CABFF28EE8CFDC
:100FE000B7F23DD00201B8517F081EE3B851B00FEF
:100FF000050DF350D06BCF6FB651CF250501C86FEB
:10100000000E0201D0210501C96F036EC851F2CF55
:10101000CAF5F29E000182EC00F00501CABFF28E13
:10102000E8CFB7F21CD00201B851A60818E3B851B6
:10103000800F050DF350D06BCF6FB651CF25050152
:10104000C86F000E0201D0210501C96FF20EC8253C
:10105000E96E010EC921EA6EEFCFB7F2020101017C
:10106000CEAF03D0FF0E0201B71BB7C2C8F5000117
:101070002DDE0201B62B93D70101CEBF05D00501AD
:10108000C86B00015DDF05D0FF0E0501C86F0001D0
:1010900057DF0201000150EF08F0C7C5B8F26AD768
:1010A000000C0501C851016AC75D03E2C7C500F025
:1010B0000CD0006A080EC96FC7370036C851005CF3
:1010C000D8B0006E0136C92FF7D70001000C0150CF
:1010D000C4C5C7F5640E0501C86F0001E2DF00C09A
:1010E000C4F50150300E08E10501C5A30ED0C5B707
:1010F0000CD0C5B9200E04D00501C597C599C5818E
:10110000012601509EA8FED7AD6EC4C5C7F50A0ED4
:10111000C86F0001C6DF00C0C4F50150300E08E101
:101120000501C5B70BD0C5A109D0C5B9200E000176
:10113000012601509EA8FED7AD6E0501300EC427D2
:10114000C4519EA8FED7AD6E0001000C1E0E050115
:10115000C46F010EC56F0001A8DD4C0E0501C76FFD
:1011600000019BDF430E0501C76F000196DF440EAF
:101170000501C76F000191DF0C0E0501C46F020E5F
:10118000C56F000192DD0301986B9851000102ECDC
:1011900001F00301982B006EE8CFC7F500017DDF59
:1011A0000A0E0301985DF1E1180E0501C46F030EEC
:1011B000C56F00017ADD0301986B9851000110ECB6
:1011C00001F00301982B006EE8CFC7F5000165DF41
:1011D000060E0301985DF1E1030E0501C46F050ED3
:1011E000C56F000162DD0301986B985100011CEC92
:1011F00001F00301982B006EE8CFC7F500014DDF29
:101200000D0E0301985DF1E184A432D00201B53DD9
:1012100003D003012DD00201010EB527C80E030132
:101220009E6F000114DD210E0501C76F000136DD40
:10123000B5C2C7F533DD0301986B985100012BEC63
:1012400001F00301982B006E00509EA8FED7AD6EF2
:10125000050E985DF2E1B5C2C4F51B0E0501C56F20
:10126000000135DF200E9EA8FED7AD6E0301CCD75E
:1012700084A233D00201B5518008D8A002D0030166
:101280002CD0010EB55FC80E03019E6F0001DFDC9C
:10129000210E0501C76F000101DDB5C2C7F5FEDCF7
:1012A0000301986B985100012BEC01F00301982B7E
:1012B000006E00509EA8FED7AD6E050E985DF2E15F
:1012C000B5C2C4F51B0E0501C56F000100DF200E7D
:1012D0009EA8FED7AD6E0301CBD7A96AB5C2A8FF01
:1012E000A69CA69EA684F2CF00F0F29E0F01550E9A
:1012F000A76EAA0EA76EA682A6B2FED7A69400502D
:10130000F212000105DDD8EF36F00501C46BC3C54C
:10131000C5F50001CADC0E0E0501C46F200EC76FB3
:101320000001BBDE0501C42FF9D70001000C808845
:10133000070E03019E6F9E3D01D008D080940000EF
:1013400000008084000000009E07F5D7000E016EAB
:101350000001000C0501F16B070EF26FF23D01D0A8
:101360001FD0F0C500F0F251016E04E0D8900032B9
:10137000012EFCD700A0809800B0808800008094E7
:10138000808480A60BD0010E006EF251016E04E045
:10139000D8900036012EFCD70050F113F207DED7AB
:1013A000F1C501F00001000CFF0E0501F06F000116
:1013B000D1DFE3C5F0F5CEDFE5C5E9F50501EA6B60
:1013C000E5C5F0F50001C6DFE4C5F0F5C3DFE7C50C
:1013D000E9F50501EA6BE7C5F0F50001BBDFE6C5FD
:1013E000F0F5B8DFE8C5F0F5B5DFFF0E0501F06FE9
:1013F0000001B0DFFF0E0501F06F0001ABDF01C09F
:10140000DFF20201DFC201F00001000C0201ED6B0E
:10141000EC6BEB6BEA6BFF0E0501F06F00019ADFDE
:101420007A0E0501F06F000195DFFF0E0501F06FE8
:10143000000190DFFF0E0501F06F00018BDFFF0E52
:101440000501F06F000186DFFF0E0501F06F00015E
:1014500081DFFF0E0501F06F00017CDFFF0E05014B
:10146000F06F000177DFFF0E0501F06F000172DF02
:10147000FF0E0501F06F00016DDF0201ED6BEC6BFB
:10148000EB6B01C0EAF2ECC2EDF2EBC2ECF2EAC2A5
:10149000EBF2EA6BFF0E0501F06F00015BDF01501C
:1014A0000201EA27000EEB23EC23ED23ECC2EDF260
:1014B000EBC2ECF2EAC2EBF2EA6BFF0E0501F06F51
:1014C000000148DF01500201EA27000EEB23EC2364
:1014D000ED23ECC2EDF2EBC2ECF2EAC2EBF2EA6B06
:1014E000FF0E0501F06F000135DF01500201EA2710
:1014F000000EEB23EC23ED23EAC200F0EBC201F077
:10150000ECC202F0EDC203F00001E0EF0AF00501C9
:101510009EBF10D00F0E006E9D3900160A0E005CA3
:1015200003E2300E002602D09E51002600509EA8F5
:10153000FED7AD6E0F0E9D170A0E9D5D02E2300EB6
:1015400002D09E9F9E519D279D519EA8FED7AD6EB5
:101550000001000C80820A0E0301986F983D01D0B3
:1015600005D00001E4DE03019807F8D78092400E11
:101570000501E36FE56BE46BE76BE66B950EE86FD7
:10158000000112DF01C099F30501C46B050EC56FA0
:10159000000155EC06F003019E6B9E51000141ECE9
:1015A00001F003019E2B006EE8CFC7F5000175DD49
:1015B0000E0E03019E5DF1E10001B9DEB8DE26D713
:1015C00003C09DF302C09CF301C09BF300C09AF3DB
:1015D0000101CEA530D003019E6B9E51000151EC5C
:1015E00001F003019E2B006E00509EA8FED7AD6E49
:1015F000060E9E5DF2E19DC39DF5570E05019E6F9F
:10160000000185DF9CC39DF5570E05019E6F00010B
:101610007EDF9BC39DF5570E05019E6F000177DFAE
:101620009AC39DF5570E05019E6F000170DF200ED5
:101630009EA8FED7AD6E03019E6B9BC39FF39CC318
:10164000A0F3A16B9E5307E19F51800804E1A03DE8
:1016500002D0A15306E0FA0E9E6F000127EC06F0BF
:1016600079D70501C46B050EC56F000155EC06F076
:1016700003019E6B9E51000141EC01F003019E2B82
:10168000006EE8CFC7F5000108DD0E0E03019E5D78
:10169000F1E1770E0501E36FE56BE46BE76BE66B59
:1016A000FF0EE86F000180DE01C099F3690E0501AD
:1016B000E36FE56BFF0EE46F800EE76FE66BFF0EE6
:1016C000E86F000171DE01C099F30101CEA51BD0C6
:1016D00003019E6B9E5100015FEC01F003019E2B04
:1016E000006E00509EA8FED7AD6E080E9E5DF2E122
:1016F00099C39DF5570E05019E6F000108DF200E6E
:101700009EA8FED7AD6E03019951050802E120D0D5
:1017100003D0995301E0BDD70501C46B050EC56F19
:10172000000155EC06F003019E6B9E5100016DEC2B
:1017300001F003019E2B006EE8CFC7F50001ADDC80
:101740000E0E03019E5DF1E18082000E016E46D017
:101750000101CEA510D003019E6B9E5100017DECCE
:1017600001F003019E2B006E00509EA8FED7AD6EC7
:10177000090E9E5DF2E1FF0E0501F06F0001EADD4A
:10178000410E0501E36FE56BE46BE76BE66BFF0E63
:10179000E86F000109DE015219E00501C46B050E76
:1017A000C56F000155EC06F003019E6B9E510001D0
:1017B0008AEC01F003019E2B006EE8CFC7F5000113
:1017C0006CDC0E0E03019E5DF1E1C2D7FF0E050138
:1017D000F06F0001BFDD010E016E0301000174EF27
:1017E00037F0E8C5F0F5B6DDEAC5EEF50501EF6BBB
:1017F000EAC5F0F50001AEDDE9C5F0F5ABDDECC5FD
:10180000EEF50501EF6BECC5F0F50001A3DDEBC5CE
:10181000F0F5A0DDEDC5F0F59DDDFF0E0501F06FE3
:10182000000198DD000C8092FF0E0501F06F0001B1
:1018300091DD500E0501E36FE56BE46BE76B010E84
:10184000E66FE86F0001B0DD015201E0EDD7FF0E59
:101850000501F06F00017EDDFF0E0501F06F000154
:1018600079DD80828092B9C5C1F5BAC5C2F505019E
:10187000B7C5C3F5B8C5C4F5510EE86FBAC5EAF5EA
:10188000B9C5E9F5B8C5ECF5B7C5EBF5010EED6FD7
:101890000001A7DFFF0E0501F06F00015BDD01C055
:1018A000BFF50501BF5303E00001F4D70501FF0EAA
:1018B000F06F00014FDD0150FE0802E00501F7D78F
:1018C000FF0E0501F06F000145DD0501BE6BBD6B2C
:1018D000BC6B01C0BBF5FF0EF06F00013BDD8082E9
:1018E000BBC500F0BCC501F0BDC502F0BEC503F02C
:1018F000000CD890DCC5DDF5DBC5DCF5DAC5DBF521
:101900000501DA6BDB37DC37DD378092FF0EF06FD5
:10191000000120DD500E0501E36FE56BE46B020E64
:10192000E76FE66BFF0EE86F00013EDD015202E05B
:101930000501ECD7FF0E0501F06F00010BDDFF0E76
:101940000501F06F000106DD80828092DCC5E4F5C0
:10195000DDC5E5F50501DAC5E6F5DBC5E7F5510EB0
:10196000E86FDDC5EAF5DCC5E9F5DBC5ECF5DAC500
:10197000EBF5010EED6F000134DFFF0E0501F06F96
:101980000001E8DC01C0E2F50501E25303E00001DB
:10199000F4D70501FF0EF06F0001DCDC0150FE08FA
:1019A000D8B402D00501F6D70501E16BE06BE15137
:1019B000010818E3DFC503F0DE51DE2BD8B4DF2BBE
:1019C000E36F03C0E4F5FF0EF06F0001C3DCE4C574
:1019D000EAFFE3C5E9FF01C0EFFF0501E02BD8B442
:1019E000E12BE5D7FF0EF06F0001B4DC8082000E22
:1019F000016E000C0501CF6BD06B010ED16FDA6A5E
:101A0000D96A050ED46FC70ED36F050EEA6ECB0EE2
:101A1000E96ED4C5E2FFD3C5E1FFD1C5D2F5D890B8
:101A2000E550EE02F350CF23F450D023D22FF7D756
:101A3000CFC5DEFFD0C5CFF5D06BD8B0D02BD32B20
:101A4000D8B4D42BD12BD1510508DFE10001000C13
:101A500005019C519E03F3CF01F0F4CF00F09F03EA
:101A6000F35000269D519E03F3500020026E0001AA
:101A7000000C006A016A026A036A0501DC6BDD6B17
:101A8000DE6BDF6BDB51DA11D911D8112CE0200E9F
:101A9000E06FD890D437D537D637D737DC37DD3736
:101AA000DE37DF37DB51DF5D08E1DA51DE5D05E16E
:101AB000D951DD5D02E1D851DC5D0FE3D851DC5F27
:101AC000D951D8A0D93DDD5FDA51D8A0DA3DDE5F2B
:101AD000DB51D8A0DB3DDF5FD8800036013602360F
:101AE0000336E02FD6D7050EEA6EDC0EE96E000154
:101AF000000C0501BA6BB96B010EB86FC90EB76F58
:101B0000000191DE03C09FF502C09EF501C09DF566
:101B100000C09CF500C0A4F50501A16BA26BA36BEE
:101B2000BA6BB96B010EB86FC80EB76F00017BDEE0
:101B300003C0A8F502C0A7F501C0A6F500C0A5F531
:101B400001C003F000C002F0006A016A0050050104
:101B5000A125AA6F0150A221AB6F0250A321AC6F47
:101B60000350A421AD6FBA6BB96B010EB86FC70EED
:101B7000B76F000158DE03C0B1F502C0B0F501C077
:101B8000AFF500C0AEF502C003F001C002F000C026
:101B900001F0006A00500501AA25B36F0150AB2186
:101BA000B46F0250AC21B56F0350AD21B66FBA6B64
:101BB000B96B010EB86FC60EB76F000134DE00506E
:101BC0000501B3250201EE6F01500501B4210201A8
:101BD000EF6F02500501B5210201F06F03500501BE
:101BE000B6210201F16F0101CEA537D005019C6B32
:101BF0009C5100019AEC01F005019C2B006E0050F5
:101C00009EA8FED7AD6E060E9C5DF2E1F1C29DF579
:101C1000570E9E6F00017BDCF0C29DF5570E05014B
:101C20009E6F000174DCEFC29DF5570E05019E6F9B
:101C300000016DDCEEC29DF5570E05019E6F00019F
:101C400066DC200E9EA8FED7AD6E0A0E9EA8FED7BB
:101C5000AD6E0D0E9EA8FED7AD6EF1C2DDF5F0C2E1
:101C6000DCF5EFC2DBF5EEC2DAF5030E0501DF6F3E
:101C70009C0EDE6F00013DDE05019E6B9D6BA8C3CF
:101C8000A2F5A16B0301A7510501A1250201F66F81
:101C9000000E0501A2210201F76F000E05019D2132
:101CA0000201F86F000E05019E210201F96F01018A
:101CB000CEA537D005019C6B9C510001A9EC01F029
:101CC00005019C2B006E00509EA8FED7AD6E070E3E
:101CD0009C5DF2E1F9C29DF5570E9E6F000117DC85
:101CE000F8C29DF5570E05019E6F000110DCF7C28A
:101CF0009DF5570E05019E6F000109DCF6C29DF5AA
:101D0000570E05019E6F000102DC200E9EA8FED733
:101D1000AD6E0A0E9EA8FED7AD6E0D0E9EA8FED724
:101D2000AD6E0201F65307E1F751020804E1F853E2
:101D300002E1F95312E005019C6B9C510001B8ECE3
:101D400001F005019C2B006E00509EA8FED7AD6EE1
:101D5000190E9C5DF2E103000201A9C3E0F201014A
:101D6000CEA523D005019C6B9C510001CDEC01F068
:101D700005019C2B006E00509EA8FED7AD6E090E8B
:101D80009C5DF2E1E0C29DF5570E9E6F000187EC6D
:101D90000AF0200E9EA8FED7AD6E0A0E9EA8FED7B2
:101DA000AD6E0D0E9EA8FED7AD6E0501ABC3A2F5BC
:101DB000A16B0301AA510501A1250201E46F000EE8
:101DC0000501A2210201E56F0101CEA52CD005017C
:101DD0009C6B9C510001DDEC01F005019C2B006E19
:101DE00000509EA8FED7AD6E060E9C5DF2E1E5C2E6
:101DF0009DF5570E9E6F000187EC0AF0E4C29DF539
:101E0000570E05019E6F000187EC0AF0200E9EA878
:101E1000FED7AD6E0A0E9EA8FED7AD6E0D0E9EA823
:101E2000FED7AD6E0101ACC3E1F2CEA523D0050112
:101E30009C6B9C510001ECEC01F005019C2B006EA9
:101E400000509EA8FED7AD6E060E9C5DF2E1E1C289
:101E50009DF5570E9E6F000187EC0AF0200E9EA89C
:101E6000FED7AD6E0A0E9EA8FED7AD6E0D0E9EA8D3
:101E7000FED7AD6E0201E451EE25F26FE551EF2180
:101E8000F36F000EF021F46F000EF121F56F0101E8
:101E9000CEA53BD005019C6B9C510001FAEC01F0F2
:101EA00005019C2B006E00509EA8FED7AD6E090E5A
:101EB0009C5DF2E1F5C29DF5570E9E6F000187EC27
:101EC0000AF0F4C29DF5570E05019E6F000187ECE4
:101ED0000AF0F3C29DF5570E05019E6F000187ECD5
:101EE0000AF0F2C29DF5570E05019E6F000187ECC6
:101EF0000AF0200E9EA8FED7AD6E0A0E9EA8FED751
:101F0000AD6E0D0E9EA8FED7AD6EF5C2CAF5F4C239
:101F1000C9F5F3C2C8F5F2C2C7F5F9C2CEF5F8C2E9
:101F2000CDF5F7C2CCF5F6C2CBF5000163DD03C0F9
:101F300005F302C004F301C003F300C002F3010182
:101F4000CEA53BD005019C6B9C5100010AEC02F030
:101F500005019C2B006E00509EA8FED7AD6E100EA2
:101F60009C5DF2E105C39DF5570E9E6F000187EC65
:101F70000AF004C39DF5570E05019E6F000187EC22
:101F80000AF003C39DF5570E05019E6F000187EC13
:101F90000AF002C39DF5570E05019E6F000187EC04
:101FA0000AF0200E9EA8FED7AD6E0A0E9EA8FED7A0
:101FB000AD6E0D0E9EA8FED7AD6E0501B3C3A2F5A2
:101FC000A16B0301B2510501A1250201E66F000ECC
:101FD0000501A2210201E76F0101CEA52BD0050169
:101FE0009C6B9C5100011EEC02F005019C2B006EC5
:101FF00000509EA8FED7AD6E070E9C5DF2E1E7C2D1
:102000009DF5570E9E6F000187EC0AF0E6C29DF524
:10201000570E05019E6F000187EC0AF0200E9EA866
:10202000FED7AD6E0A0E9EA8FED7AD6E0D0E9EA811
:10203000FED7AD6E0501AEC3A2F5A16B0301AD5194
:102040000501A1250201E86F000E0501A221020190
:10205000E96F0101CEA52BD005019C6B9C510001BD
:102060002DEC02F005019C2B006E00509EA8FED7BF
:10207000AD6E0A0E9C5DF2E1E9C29DF5570E9E6FB2
:10208000000187EC0AF0E8C29DF5570E05019E6F2E
:10209000000187EC0AF0200E9EA8FED7AD6E0A0E56
:1020A0009EA8FED7AD6E0D0E9EA8FED7AD6E0501A3
:1020B000CA6BC96BC86BE0C2C7F5F9C2CEF5F8C2EE
:1020C000CDF5F7C2CCF5F6C2CBF5000193DC03C029
:1020D00009F302C008F301C007F300C006F30201D0
:1020E000E85303E1E953D8B4D2D0E65303E1E75310
:1020F000D8B4CDD0DE91E7C29DF5E6C29CF50501CE
:102100009F6BE1C29EF50001A3DC01500201F225A4
:1021100003010E6F02500201F32103010F6F000E45
:102120000201F4210301106F000E0201F5210301E9
:10213000116F0101CEA53BD005019C6B9C510001A4
:102140003EEC02F005019C2B006E00509EA8FED7CD
:10215000AD6E0B0E9C5DF2E111C39DF5570E9E6FA7
:10216000000187EC0AF010C39DF5570E05019E6F24
:10217000000187EC0AF00FC39DF5570E05019E6F15
:10218000000187EC0AF00EC39DF5570E05019E6F06
:10219000000187EC0AF0200E9EA8FED7AD6E0A0E55
:1021A0009EA8FED7AD6E0D0E9EA8FED7AD6E0201A5
:1021B000E83505019C6F0201E93505019D6F9C37EB
:1021C0009D379C379D379C379D379C379D37E00E58
:1021D0009C17D76BD66B9DC5D5F59CC5D4F5F9C2B8
:1021E000DBF5F8C2DAF5F7C2D9F5F6C2D8F5000189
:1021F00040DC005003010E25126F01500F21136FB8
:1022000002501021146F03501121156F0101CEA54A
:102210003CD005019C6B9C5100014FEC02F0050184
:102220009C2B006E00509EA8FED7AD6E0E0E9C5DDE
:10223000F2E115C39DF5570E9E6F000187EC0AF081
:1022400014C39DF5570E05019E6F000187EC0AF03F
:1022500013C39DF5570E05019E6F000187EC0AF030
:1022600012C39DF5570E05019E6F000187EC0AF021
:10227000200E9EA8FED7AD6E0A0E9EA8FED7AD6EAC
:102280000D0E9EA8FED7AD6E0101F8D10201DE81D0
:10229000C3C3FDF20201FA6BFB6BFC6B05019D6B86
:1022A0009DC503F0C2C302F0006A016A005002013A
:1022B000FA270150FB230250FC230350FD230501A4
:1022C0009E6B9D6B9EC503F09DC502F0C1C301F0DE
:1022D000006A00500201FA270150FB230250FC2340
:1022E0000350FD23C0C300F0016A026A036A005074
:1022F000FA270150FB230250FC230350FD23010168
:10230000CEA53BD005019C6B9C51000162EC02F014
:1023100005019C2B006E00509EA8FED7AD6E0A0EE4
:102320009C5DF2E1FDC29DF5570E9E6F000187ECAA
:102330000AF0FCC29DF5570E05019E6F000187EC67
:102340000AF0FBC29DF5570E05019E6F000187EC58
:102350000AF0FAC29DF5570E05019E6F000187EC49
:102360000AF0200E9EA8FED7AD6E0A0E9EA8FED7DC
:10237000AD6E0D0E9EA8FED7AD6ECBC301F302016C
:10238000FE6BFF6B0301006B05019D6B9DC503F0A8
:10239000CAC302F0006A016A00500201FE27015020
:1023A000FF230250030100230350012305019E6B0C
:1023B0009D6B9EC503F09DC502F0C9C301F0006A84
:1023C00000500201FE270150FF23025003010023A9
:1023D00003500123016A026A036AC8510201FE2701
:1023E0000150FF2302500301002303500123010188
:1023F000CEA53BD005019C6B9C51000173EC02F013
:1024000005019C2B006E00509EA8FED7AD6E110EEC
:102410009C5DF2E101C39DF5570E9E6F000187ECB4
:102420000AF000C39DF5570E05019E6F000187EC71
:102430000AF0FFC29DF5570E05019E6F000187EC63
:102440000AF0FEC29DF5570E05019E6F000187EC54
:102450000AF0200E9EA8FED7AD6E0A0E9EA8FED7EB
:10246000AD6E0D0E9EA8FED7AD6EFDC2CAF5FCC2C4
:10247000C9F5FBC2C8F5FAC2C7F50501CE6BCD6B35
:10248000CC6BE1C2CBF50001FAEC0CF0005002017C
:10249000F22503010E6F01500201F32103010F6FBA
:1024A00002500201F4210301106F03500201F521D3
:1024B0000301116F0101CEA53BD005019C6B9C511E
:1024C00000013EEC02F005019C2B006E00509EA81E
:1024D000FED7AD6E0B0E9C5DF2E111C39DF5570E5C
:1024E0009E6F000187EC0AF010C39DF5570E0501A1
:1024F0009E6F000187EC0AF00FC39DF5570E050192
:102500009E6F000187EC0AF00EC39DF5570E050182
:102510009E6F000187EC0AF0200E9EA8FED7AD6EDC
:102520000A0E9EA8FED7AD6E0D0E9EA8FED7AD6E0C
:1025300011C3CAF510C3C9F50FC3C8F50EC3C7F55B
:10254000F9C2CEF5F8C2CDF5F7C2CCF5F6C2CBF59F
:102550000001FAEC0CF003C019F302C018F301C03B
:1025600017F300C016F30101CEA53BD005019C6B0B
:102570009C51000187EC02F005019C2B006E00507D
:102580009EA8FED7AD6E0B0E9C5DF2E119C39DF5C2
:10259000570E9E6F000187EC0AF018C39DF5570E89
:1025A00005019E6F000187EC0AF017C39DF5570ED9
:1025B00005019E6F000187EC0AF016C39DF5570ECA
:1025C00005019E6F000187EC0AF0200E9EA8FED741
:1025D000AD6E0A0E9EA8FED7AD6E0D0E9EA8FED75C
:1025E000AD6E0201E05103010E25126F000E0F21A6
:1025F000136F000E1021146F000E1121156F0101D1
:10260000CEA53CD005019C6B9C5100014FEC02F023
:1026100005019C2B006E00509EA8FED7AD6E0E0EDD
:102620009C5DF2E115C39DF5570E9E6F000187EC8E
:102630000AF014C39DF5570E05019E6F000187EC4B
:102640000AF013C39DF5570E05019E6F000187EC3C
:102650000AF012C39DF5570E05019E6F000187EC2D
:102660000AF0200E9EA8FED7AD6E0A0E9EA8FED7D9
:10267000AD6E0D0E9EA8FED7AD6E010111C30DF318
:1026800010C30CF30FC30BF30EC30AF300018AEF60
:1026900037F0030E03019B5F0AE3030EEA6E9B0E05
:1026A000E96EEF5004E001D000D0EF2EFDD700011D
:1026B000000C0301B56B070EB66FB63D01D01ED0FE
:1026C0008296B4C300F0B651016E04E0D890003297
:1026D000012EFCD700A0829A00B0828A828682A84E
:1026E0000BD0010E006EB651016E04E0D89000369A
:1026F000012EFCD70050B513B607DFD7B5C301F0E4
:102700000001000C0301AE6BAF6BB06BB16BB26B31
:10271000B36B8294AAC3B4F30001CBDFABC3B4F3B1
:10272000C8DFACC3B4F3C5DF0301AF6B01C0AEF3C8
:10273000ADC3B4F30001BDDF0301B16B01C0B0F361
:10274000B46BB451B011B26FAE51B111B36F82849A
:10275000B2C301F0B3C302F00001000C8284819C7B
:10276000020E0301986FF90E9B6F000192DF0301C7
:10277000982FF9D7818C020E986FF90E9B6F00018C
:1027800088DF0301982FF9D7020EAA6F0B0EAB6FEB
:10279000A00EAC6FAD6F0001B5DF020E0301AA6F92
:1027A000030EAB6F300EAC6FD40EAD6F0001AADF1D
:1027B000280E0101DD6F020E0301AA6F0B0EAB6F35
:1027C000DDC1ACF3DDC1ADF300019CDFA0EF37F05C
:1027D000E9500501CC6F3B0ED36F9A0ED26FCA0E33
:1027E000D16FD06B0A0ECE6FCBC5D7F5CAC5D6F563
:1027F000C9C5D5F5C8C5D4F5D3C5DBF5D2C5DAF55D
:10280000D1C5D9F5D0C5D8F5000139EC0DF001508E
:10281000EFCFC8F5ECCFC9F5ECCFCAF5ECCFCBF5CF
:10282000005213E10501CE51010AD8A402D00001E3
:102830000CD0CC510CE00F0BCE5D01E00EE2CCBF12
:102840000CD0CCBD04D0200E03D00501CC6B300ED3
:10285000002600509EA8FED7AD6ED3C5D7F5D2C5D1
:10286000D6F5D1C5D5F5D0C5D4F5DB6BDA6BD96B10
:102870000A0ED86F000139EC0DF003C0D3F502C089
:10288000D2F501C0D1F500C0D0F50501CE2FACD7EF
:102890000001000C0150C5C5C7F5640E0501C86FE5
:1028A000000151EC08F000C0C5F50150300E08E100
:1028B0000501C6A310D0C6B70ED0C6B9200E04D0ED
:1028C0000501C697C699C681012601C0C7F500015A
:1028D0004DEC08F00501C5C5C7F50A0EC86F00012B
:1028E00051EC08F000C0C5F50150300E08E10501BB
:1028F000C6B70BD0C6A109D0C6B9200E000101266B
:1029000001C0C7F54DEC08F00501300EC527C5C55F
:10291000C7F500014DEC08F0000CEACFCBF5E9CF8C
:10292000CAF50501C439F009C66FC627E20FC76FA3
:10293000320FC96FC4510F0BC727C727C927E90F2B
:10294000C86FC827C827C3390F0BC827C927C8377E
:10295000C937C91FC937C3510F0BC927C637070E5F
:10296000C56F0A0EC807C927FDE3C707C827FDE3DF
:10297000C607C727FDE3C507C627FDE3050EEA6EB8
:10298000C50EE96E070ECA15CA9DE926C90EE95C97
:10299000D8B4CA8DEF50006E08E1CABD06D0CAB9DE
:1029A0000CD0CAB702D0200E03D0CA87CA99300E05
:1029B000002600509EA8FED7AD6EEE50CAADE6D7F9
:1029C0000001000C0501B96B0101D96BD86BCF6B0D
:1029D000D06B0501A56BA46BA36BA26B0101D46B3B
:1029E0000301982D22D00501C46B050EC56F0001AF
:1029F00055EC06F00501C36BC351000198EC02F0E1
:102A00000501C32B006EC76F00014DEC08F0080EE6
:102A10000501C35DF1E1040EC46F2E0EC76F000106
:102A20004DEC08F00501C42FF8D70201DEA110D04B
:102A3000F5C2A1F5F4C2A0F5F3C29FF5F2C29EF56E
:102A400001C3A9F500C3A8F5FFC2A7F5FEC2A6F50C
:102A500011C3B8F510C3B7F50FC3B6F50EC3B5F57E
:102A60000501B16BB06BAF6BAE6B0201DEA10FD095
:102A7000E0510501B525BF6F000EB621C06F000EF5
:102A8000B721C16F000EB821C26F32D00201DEB192
:102A90002FD0E8350501C36F0201E9350501C46F88
:102AA000C337C437C337C437C337C437C337C43752
:102AB000E00EC317D76BD66BC4C5D5F5C3C5D4F527
:102AC000F9C2DBF5F8C2DAF5F7C2D9F5F6C2D8F5E6
:102AD000000139EC0DF000500501B525BF6F015024
:102AE000B621C06F0250B721C16F0350B821C26F29
:102AF000B8C59DF5B7C59CF5B6C59BF5B5C59AF5A6
:102B00000501BF519A5D0BE1C0519B5D08E1C151C8
:102B10009C5D05E1C2519D5DD8B431EF1BF0C36BE4
:102B2000C3510001A5EC02F00501C32B006E00505B
:102B30009EA8FED7AD6E0A0EC35DF2E1410EE96EAE
:102B40009DC5CBF59CC5CAF59BC5C9F59AC5C8F509
:102B500000013EDE200E9EA8FED7AD6E0501C36BC0
:102B6000C3510001B5EC02F00501C32B006E00500B
:102B70009EA8FED7AD6E080EC35DF2E1410EE96E70
:102B8000ADC5CBF5ACC5CAF5ABC5C9F5AAC5C8F589
:102B900000011EDE200E9EA8FED7AD6E0501C36BA0
:102BA000C3510001C4EC02F00501C32B006E0050BC
:102BB0009EA8FED7AD6E090EC35DF2E1410EE96E2F
:102BC000B1C5CBF5B0C5CAF5AFC5C9F5AEC5C8F539
:102BD0000001FEDD200E9EA8FED7AD6E0501B951A5
:102BE000040DF350036A400FE96E010E0320EA6EF4
:102BF000EFCFC3F5ECCFC4F5ECCFC5F5ECCFC6F500
:102C0000C76BC7510001D3EC02F00501C72B006E62
:102C100000509EA8FED7AD6E090EC75DF2E1410ED1
:102C2000E96EC6C5CBF5C5C5CAF5C4C5C9F5C3C5EA
:102C3000C8F50001CDDD0A0E9EA8FED7AD6E0D0EC3
:102C40009EA8FED7AD6E0501AA530BE1AB51020859
:102C500008E1AC5306E1AD5304E1B16BB06BAF6B6F
:102C6000AE6B9DC5DDF59CC5DCF59BC5DBF59AC556
:102C7000DAF5030EDF6F9A0EDE6F000179EC0CF0CF
:102C8000B1C5ADF5B0C5ACF5AFC5ABF5AEC5AAF5F0
:102C90000501AA5309E1AB51020806E1AC5304E176
:102CA000AD53D8B427EF1BF09A0EAA25E96E030E98
:102CB000AB21EA6EEF507F0812E2C36BC3510001F3
:102CC000E3EC02F00501C32B006E00509EA8FED776
:102CD000AD6E040EC35DF2E11FEF1BF001D30B0ECE
:102CE000AA25C36F000EAB21C46F000EAC21C56FC7
:102CF000000EAD21C66F9A0EC325E96E030EC421E6
:102D0000EA6EEF500C0B0C0812E1C36BC3510001CB
:102D1000EEEC02F00501C32B006E00509EA8FED71A
:102D2000AD6E040EC35DF2E11FEF1BF0D9D29A0E17
:102D3000AA25E96E030EAB21EA6EEF52D8A47AD031
:102D4000B951000863E2C36BC3510001F9EC02F012
:102D50000501C32B006E00509EA8FED7AD6E050E78
:102D6000C35DF2E1B907010E0101D0270501B95198
:102D7000040DF350036A400FE96E010E0320EA6E62
:102D8000EFCF00F0ECCF01F0ECCF02F0ECCF03F08E
:102D900003C0B1F502C0B0F501C0AFF500C0AEF59B
:102DA000B951040DF350036A680FE96E010E032058
:102DB000EA6EEFCF00F0ECCF01F0ECCF02F0ECCFF9
:102DC00003F003C0B8F502C0B7F501C0B6F500C006
:102DD000B5F5200EAE27000EAF23B023B123AE53BE
:102DE00013E1AF51020810E1B0530EE1B1530CE111
:102DF000010EB527D8B0B62BD8B4B72BD8B4B82BA2
:102E0000B16BB06BAF6BAE6B30D613D0B95311E171
:102E1000C36BC351000104EC03F00501C32B006E2A
:102E200000509EA8FED7AD6E050EC35DF2E1A2EF85
:102E30001EF056D20B0EAA25C36F000EAB21C46F35
:102E4000000EAC21C56F000EAD21C66F9A0EC325D2
:102E5000E96E030EC421EA6EEF501C0B1008D8A4D3
:102E6000D1D19A0EAA25E96E030EAB21EA6EEF507E
:102E70002E0802E11FEF1BF00301985304E101014A
:102E8000D52B16D003019851020812E10101D42B71
:102E9000D451D35D0DE1010ED825DA6F000ED92192
:102EA000DB6FCE9B010E0301986F00018BD50101F2
:102EB0000501B951040DF350036A400FE96E010E8C
:102EC0000320EA6EAAC5EFFFABC5ECFFACC5ECFF73
:102ED000ADC5ECFFB951040DF350036A680FE96EFC
:102EE000010E0320EA6E9AC5EFFF9BC5ECFF9CC55F
:102EF000ECFF9DC5ECFFB92B0101CF2B036ACF512D
:102F0000A90FE96E010E0320EA6EB9C5EFFFD06B81
:102F1000030198510308D8A4C2D00101D35302E1A0
:102F2000010ED36FD42BD351D45DD8A08ED0050120
:102F3000B95100083DE2020EEA6ED10EE96EF2CF01
:102F4000C3F5F29E000E000138EC01F00A00090002
:102F5000F550EE6E0009FBE10501C3BFF28E0301DF
:102F6000996B9951080823E0036A9951D10F016EBA
:102F7000020E0322030199510501AA25C56F000E17
:102F8000AB21C66F000EAC21000EAD219A0EC525F7
:102F9000E96E030EC621EA6EEFCFC9F503C0EAFF62
:102FA00001C0E9FFC9C5EFFF0301992BDAD705017D
:102FB000C46BDCC1C5F5000155EC06F00101DC5322
:102FC000D8B4CE8FDC51D325036A900FE96E010E81
:102FD0000320EA6EEFCFC4F5C4C5C5F5130E050195
:102FE000C66F000157DC200E0501C76F00014DECD4
:102FF00008F0B9C5BAF50501BA5308E02E0EC76F3F
:1030000000014DEC08F00501BA07F6D75C0EC76F5A
:1030100000014DEC08F0020EEA6ED10EE96E000ED2
:10302000EF1010E0EACFC4F5E9CFC3F5EFCFC7F555
:103030004DEC08F0C4C5EAFFC3C5E9FFE92AD8B4DE
:10304000EA2AEDD70101CE9FDC2B030ED325D45DF8
:1030500003E0D551D45D22E10501C46B040EC56FB8
:10306000000155EC06F00501C36BC35100010FECE4
:1030700003F00501C32B006EC76F00014DEC08F093
:10308000080E0501C35DF1E190C1C5F51B0EC66FC9
:10309000000100DC0501A2EF1EF001010301982DE3
:1030A00002D0CFC1D3F1150E0501AA25C36F000EC2
:1030B000AB21C46F000EAC21000EAD219A0EC325CA
:1030C000E96E030EC421EA6EEF50C76FCC6BCD6B77
:1030D000CE6B140EAA25D06F000EAB21D16F000E5F
:1030E000AC21000EAD219A0ED025E96E030ED12140
:1030F000EA6EEF50D56BD46F006A016A0050CC25A0
:10310000BB6F0150CD21BC6FD451CE21BD6FD551C5
:10311000C721BE6F1B0EAA25C36F000EAB21C46F63
:10312000000EAC21000EAD219A0EC325E96E030EF0
:10313000C421EA6EEF50C96BC86BC76FCC6B1A0E17
:10314000AA25D06F000EAB21D16F000EAC21000E6E
:10315000AD219A0ED025E96E030ED121EA6EEF5013
:10316000CC25006E000EC721016E000EC821026E34
:10317000000EC921036E0050BB270150BC23025032
:10318000BD230350BE23020EBB5F000EBC5BBD5BC4
:10319000BE5BBEC5CAF5BDC5C9F5BCC5C8F5BBC5D6
:1031A000C7F5CE6BCD6BCC6BE0C2CBF50001FAEC72
:1031B0000CF003C0B8F502C0B7F501C0B6F500C009
:1031C000B5F5030112510501B5270301135105019E
:1031D000B623030114510501B7230301155105015D
:1031E000B8230201DEA107D0E0510501B55F000E52
:1031F000B65BB75BB85B0501B16BB06BAF6BAE6B29
:1032000034D46ED003019853D8A46BD0030E0501BB
:10321000C36F2A0E9EA8FED7AD6EC32FFAD7C46B1C
:10322000C45100011DEC03F00501C42B006E0050D9
:103230009EA8FED7AD6E060EC45DF2E1100EE96EDB
:10324000D7C1C4F5D6C1C3F500018DEC14F0200E32
:103250009EA8FED7AD6E0501C36BC351000129ECDA
:1032600003F00501C32B006E00509EA8FED7AD6E83
:103270000B0EC35DF2E1CFC1C4F51B0EC56F00019B
:1032800067EC08F0200E9EA8FED7AD6E0501B9537D
:1032900021E00101D0530FE0D051CF5D036AA90FA7
:1032A000E96E010E0320EA6EEF500501B95D04E2FC
:1032B0000101D02BF1D705010101D051CF5D036A87
:1032C000900FE96E010E0320EA6E010EEF24EF6EFF
:1032D00006D00501B95304E1010E01019027050153
:1032E0000301080E0501AA25C36F000EAB21C46FB0
:1032F000000EAC21000EAD219A0EC325E96E030E1F
:10330000C421EA6EEFCFB2F5090EAA25C36F000EF5
:10331000AB21C46F000EAC21000EAD219A0EC32567
:10332000E96E030EC421EA6EEFCFB3F50A0EAA25AB
:10333000C36F000EAB21C46F000EAC21000EAD2197
:103340009A0EC325E96E030EC421EA6EEFCFB4F5E1
:10335000B2516D0804E0B2514D08D8A470D1B351F8
:10336000500804E0B3517008D8A469D1B4513308AF
:10337000D8A465D10301985306E10101D62BD8B436
:10338000D72B5BD10301982D51D10101D82BD8B493
:10339000D92BD851DA5DD8A447D1D951DB5DD8A457
:1033A00043D1050E0501C36F000185EC09F0150E30
:1033B0000501AA25C36F000EAB21C46F000EAC211E
:1033C000000EAD219A0EC325E96E030EC421EA6EEC
:1033D000EF50C76FCC6BCD6BCE6B140EAA25D06FA0
:1033E000000EAB21D16F000EAC21000EAD219A0E64
:1033F000D025E96E030ED121EA6EEF50D56BD5C50D
:1034000003F0026E006A016A0050CC2503011E6FB2
:1034100001500501CD2103011F6F02500501CE218E
:103420000301206F03500501C7210301216F1B0E0B
:103430000501AA25C36F000EAB21C46F000EAC219D
:10344000000EAD219A0EC325E96E030EC421EA6E6B
:10345000EF50C96BC86BC76FCC6B1A0EAA25D06F23
:10346000000EAB21D16F000EAC21000EAD219A0EE3
:10347000D025E96E030ED121EA6EEF50CC25006E07
:10348000000EC721016E000EC821026E000EC92178
:10349000036E005003011E2701501F2302502023FA
:1034A00003502123020E1E5D0501C36F000E0301B0
:1034B0001F590501C46F000E030120590501C56F96
:1034C000000E030121590501C66FCA6FC5C5C9F5B4
:1034D000C4C5C8F5C3C5C7F5CE6BCD6BCC6BE0C218
:1034E000CBF50001FAEC0CF003C0C5F102C0C4F149
:1034F00001C0C3F100C0C2F1030112510101C22792
:10350000030113510101C323030114510101C42319
:10351000030115510101C5230201DEA107D0E051CD
:103520000101C25F000EC35BC45BC55B1F0E0501DA
:10353000AA25C36F000EAB21C46F000EAC21000E94
:10354000AD219A0EC325E96E030EC421EA6EEF5039
:10355000C76FCC6BCD6BCE6B1E0EAA25D06F000E45
:10356000AB21D16F000EAC21000EAD219A0ED025FB
:10357000E96E030ED121EA6EEF50D56BD5C503F08D
:10358000026E006A016A0050CC250301226F0150CF
:103590000501CD210301236F02500501CE21030156
:1035A000246F03500501C7210301256F1D0E05017E
:1035B000AA25C36F000EAB21C46F000EAC21000E14
:1035C000AD219A0EC325E96E030EC421EA6EEF50B9
:1035D000C96BC86BC76FCC6B1C0EAA25D06F000ED1
:1035E000AB21D16F000EAC21000EAD219A0ED0257B
:1035F000E96E030ED121EA6EEF50CC25006E000E6D
:10360000C721016E000EC821026E000EC921036E93
:10361000005003012227015023230250242303508A
:10362000252305018FD3010108D003019851020819
:1036300005E10101D82BD8B4D92B03010501200ED7
:10364000AA27000EAB23AC23AD2349EF16F0010EE1
:103650009A27D8B09B2BD8B49C2BD8B49D2B81EF44
:1036600015F0200E9EA8FED7AD6E040EC36F2A0E75
:103670009EA8FED7AD6EC32FFAD7200E9EA8FED708
:10368000AD6E03010A510501B55DC36F03010B5116
:103690000501B659C46F03010C510501B759C56F37
:1036A00003010D510501B859C66FD8900201E035EC
:1036B0000501C325C76F000EC421C86F000EC521C8
:1036C000C96F000EC621CA6FD76FC9C5D6F5C8C568
:1036D000D5F5C7C5D4F5DB6BDA6BD96BE0C2D8F58D
:1036E000000139EC0DF003C0A9F502C0A8F501C036
:1036F000A7F500C0A6F50201DEB13AD0D890F931A5
:10370000036EF831026EF731016EF631006E03C0C0
:10371000C6F502C0C5F501C0C4F5E8CFC3F5A9C51B
:10372000D7F5A8C5D6F5A7C5D5F5A6C5D4F503C068
:10373000DBF502C0DAF501C0D9F5E8CFD8F5000114
:1037400039EC0DF00201F251050100249E6F0201D7
:10375000F351050101209F6F0201F4510501022080
:10376000A06F0201F55105010320A16F40D00201B5
:10377000DEA13DD0F931036EF831026EF731016EF2
:10378000F631006E03320232013200323F0E031670
:1037900003C0C6F502C0C5F501C0C4F500C0C3F53D
:1037A000A9C5D7F5A8C5D6F5A7C5D5F5A6C5D4F53D
:1037B00003C0DBF502C0DAF501C0D9F500C0D8F5C9
:1037C000000139EC0DF00201F251050100249E6F59
:1037D0000201F351050101209F6F0201F45105011F
:1037E0000220A06F0201F55105010320A16F050120
:1037F000C36BC351000139EC03F00501C32B006E0C
:1038000000509EA8FED7AD6E0F0EC35DF2E1080E0C
:10381000E96EA9C5CBF5A8C5CAF5A7C5C9F5A6C562
:10382000C8F50001E8EC13F0200E9EA8FED7AD6E9F
:103830000A0E9EA8FED7AD6E0D0E9EA8FED7AD6EE9
:103840000201DEB1FCD0A1C5DDF5A0C5DCF59FC548
:10385000DBF59EC5DAF5030E0501DF6F9A0EDE6F0C
:10386000000179EC0CF00501006A0050A65DC76FFD
:10387000A751A759C86FA851A859C96FA951A959EB
:10388000CA6FD890C735AA6FC835AB6FC935AC6F52
:10389000CA35AD6F010EAA25C36F000EAB21C46FF0
:1038A000000EAC21000EAD219A0EC325E96E030E69
:1038B000C421EA6EEF50C96BC86BC76FCC6B9A0E10
:1038C000AA25E96E030EAB21EA6EEF50CC25A26F5C
:1038D000000EC721A36F000EC821A46F000EC921DE
:1038E000A56FA5530CE1A4530AE1A351FE08D8B07B
:1038F000A4D0FF0A04E1A251EF08D8B09ED0C36B58
:10390000C35100014DEC03F00501C32B006E0050C4
:103910009EA8FED7AD6E0C0EC35DF2E1080EE96EF7
:10392000A5C5CBF5A4C5CAF5A3C5C9F5A2C5C8F5FB
:103930000001E8EC13F0200E9EA8FED7AD6E0A0E33
:103940009EA8FED7AD6E0D0E9EA8FED7AD6ED89088
:103950000201F931036EF831026EF731016EF63172
:10396000006E03C0C6F502C0C5F501C0C4F5E8CFBE
:10397000C3F5A5C5D7F5A4C5D6F5A3C5D5F5A2C58C
:10398000D4F503C0DBF502C0DAF501C0D9F5E8CF04
:10399000D8F5000139EC0DF00201F25105010024C7
:1039A0009E6F0201F351050101209F6F0201F45146
:1039B00005010220A06F0201F55105010320A16F4E
:1039C000A5C5A9F5A4C5A8F5A3C5A7F5A2C5A6F5E3
:1039D000A9C5CAF5A8C5C9F5A7C5C8F5A6C5C7F53F
:1039E000CE6BCD6BCC6BE0C2CBF50001FAEC0CF0EA
:1039F00003010A5105010024C76F03010B510501A2
:103A00000120C86F03010C5105010220C96F030199
:103A10000D5105010320CA6FD8900201E035050160
:103A2000C75DB56F000EC859B66F000EC959B76FA4
:103A3000000ECA59B86F35EF15F084D10201DEA12E
:103A400082D1A1C5DDF5A0C5DCF59FC5DBF59EC51E
:103A5000DAF5030E0501DF6F9A0EDE6F000179ECD7
:103A60000CF00501A931C66FA831C56FA731C46F2D
:103A7000A631C36FC633C533C433C333C633C5336E
:103A8000C433C333C633C533C433C333C633C5337A
:103A9000C433C333C633C533C433C333C633C5336A
:103AA000C433C333010EC617C335006EC435016E6F
:103AB000C535026EC635036E003601360236033652
:103AC000003601360236033600360136023603363A
:103AD000003601360236033600360136023603362A
:103AE0000036013602360336800E00160050A65D01
:103AF000C76F0150A759C86F0250A859C96F03502A
:103B0000A959CA6FC735AA6FC835AB6FC935AC6F35
:103B1000CA35AD6FAA37AB37AC37AD37FC0EAA1735
:103B2000030EAA25C36F000EAB21C46F000EAC219B
:103B3000000EAD219A0EC325E96E030EC421EA6E74
:103B4000EF50C76FCC6BCD6BCE6B020EAA25D06F3A
:103B5000000EAB21D16F000EAC21000EAD219A0EEC
:103B6000D025E96E030ED121EA6EEF50D56BD46FEC
:103B7000006A016A0050CC25A26F0150CD21A36FCD
:103B8000D451CE21A46FD551C721A56F010EAA250E
:103B9000C36F000EAB21C46F000EAC21000EAD212F
:103BA0009A0EC325E96E030EC421EA6EEF50C96B6D
:103BB000C86BC76FCC6B9A0EAA25E96E030EAB21BA
:103BC000EA6EEF50CC25006E000EC721016E000E8C
:103BD000C821026E000EC921036E0050A2270150B9
:103BE000A3230250A4230350A523A23D08D0A33D44
:103BF00006D0A43D04D0A5510F08D8B4A3D0C36B00
:103C0000C35100014DEC03F00501C32B006E0050C1
:103C10009EA8FED7AD6E0C0EC35DF2E1080EE96EF4
:103C2000A5C5CBF5A4C5CAF5A3C5C9F5A2C5C8F5F8
:103C30000001E8EC13F0200E9EA8FED7AD6E0A0E30
:103C40009EA8FED7AD6E0D0E9EA8FED7AD6E0201EA
:103C5000F931036EF831026EF731016EF631006E04
:103C600003320232013200323F0E031603C0C6F5A2
:103C700002C0C5F501C0C4F500C0C3F5A5C5D7F5A0
:103C8000A4C5D6F5A3C5D5F5A2C5D4F503C0DBF50B
:103C900002C0DAF501C0D9F500C0D8F5000139EC51
:103CA0000DF00201F251050100249E6F0201F35153
:103CB000050101209F6F0201F45105010220A06F50
:103CC0000201F55105010320A16FA5C5A9F5A4C501
:103CD000A8F5A3C5A7F5A2C5A6F5A9C5CAF5A8C5A7
:103CE000C9F5A7C5C8F5A6C5C7F5CE6BCD6BCC6B1E
:103CF000E0C2CBF50001FAEC0CF003010A5105011A
:103D00000024C76F03010B5105010120C86F030197
:103D10000C5105010220C96F03010D51050103205B
:103D2000CA6FD8900201E0350501C75DB56F000E7E
:103D3000C859B66F000EC959B76F000ECA59B86F8F
:103D400035EF15F002010001000C9DC30AF09CC381
:103D500009F09BC308F09AC307F0F9EF37F0016A46
:103D6000026A006A036A03019E5102E19D5118E054
:103D7000100E9F6FD8909B379C37003603369E51AC
:103D8000035C02E19D51005C07E39D51005ED8A0F9
:103D900003069E51035ED880013602369F2FEAD774
:103DA000000108EF1FF00AC0CAF509C0C9F508C034
:103DB000C8F507C0C7F5410E0501CE6FC60ECD6F21
:103DC0004E0ECC6F6D0ECB6F0001FAEC0CF0390E7D
:103DD00003010024076E300E0120086E000E022041
:103DE000096E000E03200A6E09C000F00AC001F03F
:103DF000026A036A0AC09AF309C099F30AC09CF3E5
:103E000009C09BF3030E9E6FE70E9D6F0001A7D7BD
:103E100000C001F003C002F0FDEF30F00501C36BFC
:103E2000000185EC09F0010E0501C36F000185EC6E
:103E300009F0020E0501C36F000185EC09F0030EC5
:103E40000501C36F000185EC09F0040E0501C36F85
:103E5000000185EC09F0050E0501C36F000185EC3A
:103E600009F0000C8188070E03019B6F9B3D01D078
:103E700012D09AC300F09B51016E04E0D89000323A
:103E8000012EFCD700A0819600B0818681848194A8
:103E900081989B07EBD70001000C0301996B986B8D
:103EA000985303E1995108080AE081A2FED79A6B62
:103EB0000001D8DF0301982BD8B4992BF1D7020E5B
:103EC000AA6FAB6B010EAC6F040EAD6F000182ECFC
:103ED00013F0100E006E002EFED7000081B201D04C
:103EE000FDD7020E03019A6FC70E9B6F000149ECCC
:103EF00013F003019A2FF8D79A6B0001B3DF030187
:103F00009A6B0001AFDF15EF31F00301D86B87C367
:103F1000DDF586C3DCF585C3DBF584C3DAF5030E76
:103F20000501DF6FDA0EDE6F000179EC0CF00301A2
:103F3000D96BD951F90833E3DA0ED925E96E030EAE
:103F4000EA6ED8B0EA2AEF501F0822E209D0DA0E52
:103F5000D925E96E030EEA6ED8B0EA2A00A018D07F
:103F6000036AD851D625016ED7510322DA0E030118
:103F7000D925E96E030EEA6ED8B0EA2AEFCFDCF558
:103F800003C0EAFF01C0E9FFDCC5EFFF0301D82B46
:103F9000D851F80802E2FA0ED96FD92BCAD7D851F6
:103FA000F9080BE3036AD851D625E96ED7510320EF
:103FB000EA6E200EEF6ED82BF2D700015EEF25F0EF
:103FC000ECC303F00301EBC3E9FFECC3EAFFEF52DC
:103FD00039E0ECC3F0F3EBC3EFF3EEC3F2F3EDC360
:103FE000F1F3F2C303F0F1C3E9FFF2C3EAFFEF52CA
:103FF00016E0EFC3E9FFF0C3EAFFEFCFF3F3F2C33C
:1040000003F0F1C3E9FFF2C3EAFFEF50F35D07E10C
:10401000EF2BD8B4F02BF12BD8B4F22BE2D7F2C3AC
:1040200003F0F1C3E9FFF2C3EAFFEF5205E1EBC38E
:1040300001F0ECC302F009D0EB2BD8B4EC2B00015B
:10404000BFD70301000E016E026E0001000CECC32D
:10405000EEF3EBC3EDF3EEC303F00301EDC3E9FFB1
:10406000EEC3EAFFEF5206E0ED2BD8B4EE2B0001D1
:10407000F2D70301EB51ED5D006EEC51EE59036E8A
:1040800000C001F0026E0001000C0301EC6B0B0E8E
:10409000EB6F030EEE6F330EED6F000191DF01C089
:1040A0005AF30301EC6B0B0EEB6F030EEE6F2E0E4B
:1040B000ED6F000185DF01C059F30301EC6B0B0EBE
:1040C000EB6F030EEE6F420EED6F000179DF01C062
:1040D00057F30301EC6B0B0EEB6F030EEE6F380E14
:1040E000ED6F00016DDF01C056F30301EC6B0B0EA9
:1040F000EB6F030EEE6F3D0EED6F000161DF01C04F
:104100005CF30301EC6B0B0EEB6F030EEE6F470ECF
:10411000ED6F000155DF01C058F30301EC6B0B0E8E
:10412000EB6F030EEE6F4C0EED6F000149DF01C027
:104130005BF30301EC6B0B0EEB6F030EEE6F510E96
:10414000ED6F00013DDF01C05DF30301EC6B0B0E71
:10415000EB6F00017CDF01C066F30301EC6B5AC317
:10416000EBF3000174DF01C068F30301EC6B59C38A
:10417000EBF300016CDF01C067F30301EC6B57C385
:10418000EBF3000164DF01C06AF30301EC6B56C37B
:10419000EBF300015CDF01C069F30301EC6B5CC36E
:1041A000EBF3000154DF01C06DF30301EC6B58C366
:1041B000EBF300014CDF01C06BF30301EC6B5BC35D
:1041C000EBF3000144DF01C06CF30301EC6B5DC352
:1041D000EBF300013CDF01C06EF368C3DAF367C3A1
:1041E000DBF36AC3DCF369C3DDF36DC3DEF36BC3DA
:1041F000DFF36CC3E0F36EC3E1F30301EC6B5AC36E
:10420000EBF3000124DF01500301665D626FEC6B8C
:1042100059C3EBF300011BDF01500301665D616FC1
:10422000EC6B57C3EBF3000112DF01500301665D35
:104230005F6FEC6B56C3EBF3000109DF0150030124
:10424000665D5E6FEC6B5CC3EBF3000100DF015059
:104250000301665D646FEC6B58C3EBF30001F7DE9E
:1042600001500301665D606FEC6B5BC3EBF3000113
:10427000EEDE01500301665D636FEC6B5DC3EBF333
:104280000001E5DE01500301665D656FD66BD76BFB
:10429000D73D01D022D0D86BD851070816E3036A66
:1042A000D851DA0FE96E030E0320EA6ED751EF5CA6
:1042B0000AE1036AD651E30FE96E030E0320EA6EAA
:1042C000D8C3EFFFD62BD82BE7D7D651080803E188
:1042D000FF0ED76F02D0D72BDBD7EC6B5AC3EBF3B3
:1042E0000001B5DE01C068F3070E0301D96FD95391
:1042F00023E0036AD951E30FE96E030E0320EA6E4F
:10430000EF5218E1D953D8A4D907D9C3D6F3036A19
:10431000D651E30FE96E030E0320EA6EEFCFE2F30E
:10432000036AE251DA0FE96E030E0320EA6EEF50E2
:10433000685F02D0D907DBD7EC6B59C3EBF3000100
:1043400086DE01C067F3070E0301D96FD95323E05E
:10435000036AD951E30FE96E030E0320EA6EEF2CD6
:1043600018D0D953D8A4D907D9C3D6F3036AD651E4
:10437000E30FE96E030E0320EA6EEFCFE2F3036A68
:10438000E251DA0FE96E030E0320EA6EEF50675F29
:1043900002D0D907DBD7040E685F675F68511B083E
:1043A00002E21C0E686F67511B0802E21C0E676F69
:1043B000000160EF25F0E1C3E6F3E0C3E5F303019C
:1043C000E45324E0E3C303F0E2C3E9FFE3C3EAFFFD
:1043D000EF521CE0E6C303F0E551E52BD8B4E62B21
:1043E000E76F03C0E8F3E3C303F0E251E22BD8B474
:1043F000E32BE96E03C0EAFFEFCFE9F3E8C3EAFF7E
:10440000E7C3E9FFE9C3EFFFE407DAD7E4530CE0C1
:10441000E6C303F0E551E52BD8B4E62BE96E03C003
:10442000EAFFEF6AE407F2D7E0C301F0E1C302F06C
:104430000001000C0301D86BD76B67511B0857E2D2
:104440000B0E6125D96FDA6BD8B0DA2B040ED925A3
:10445000DB6F000EDA21DC6F010EE16F060EE06FFC
:10446000DCC3E3F3DBC3E2F367C3E4F30001A3DFE0
:104470001B0E0301D66FD651010810E2036AD65114
:10448000060FE96E010E0320EA6EEF50200803E0EC
:10449000010E675F01D002D0D607EDD71B0ED66F95
:1044A000D651010810E2036AD651060FE96E010EDB
:1044B0000320EA6EEF50200803E1010E675F01D090
:1044C00002D0D607EDD7010EEA6E060EE96EF2CFE6
:1044D000D9F3F29E000E0001B7EC03F00A000900C8
:1044E000F550EE6E0009FBE10301D9BFF28E675172
:1044F0000E0826E30E0ED8806755006ED890003265
:104500000050060FDA6F010EDB6FD8B0DB2B0B0EFD
:104510006125DC6FDD6BD8B0DD2B040EDC25DE6F92
:10452000000EDD21DF6FDBC3E1F3DAC3E0F3E36FFD
:10453000DEC3E2F367C3E4F300013DDF86D003018D
:1045400067511B08D8A082D00B0E6125D96FDA6B9A
:10455000D8B0DA2B040ED925DB6F000EDA21DC6F20
:10456000010EE16F060EE06FDCC3E3F3DBC3E2F3A1
:1045700067C3E4F300011FDF0E0E0301D66FD651AF
:10458000010810E2036AD651060FE96E010E0320FE
:10459000EA6EEF50200804E1D6C3D8F3010ED66FBF
:1045A000D607EDD7D851675DD76FD7510E0802E215
:1045B0000E0ED76F010EEA6E060EE96EF2CFD9F33A
:1045C000F29E000E0001B7EC03F00A000900F5505E
:1045D000EE6E0009FBE10301D9BFF28E0B0E6125DF
:1045E000D96FDA6BD8B0DA2B040ED925DB6F000E49
:1045F000DA21DC6F010EE16F060EE06FDCC3E3F33E
:10460000DBC3E2F3D8C3E4F30001D5DE0B0E0301F4
:104610006125D96FDA6BD8B0DA2B040ED925DB6FA0
:10462000000EDA21DC6FD851DB25DD6F000EDC21B6
:10463000DE6F010EE16F140EE06FDEC3E3F3DDC346
:10464000E2F3D7C3E4F30001B6DE03016151EF08E2
:1046500014E2010EEA6E060EE96EF2CFD9F3F29E75
:10466000000E00010EEC04F00A000900F550EE6E99
:104670000009FBE10301D9BFF28ED86BD76B6851FB
:104680001B08D8B06CD00B0E6225D96FDA6BD8B08E
:10469000DA2B040ED925DB6F000EDA21DC6F010E58
:1046A000E16F230EE06FDCC3E3F3DBC3E2F368C327
:1046B000E4F3000180DE1B0E0301D66FD651010822
:1046C00010E2036AD651230FE96E010E0320EA6E51
:1046D000EF50200803E0010E685F01D002D0D6073A
:1046E000EDD71B0ED66FD651010810E2036AD651E2
:1046F000230FE96E010E0320EA6EEF50200803E15C
:10470000010E685F01D002D0D607EDD71C0ED66F20
:10471000D651010810E2036AD651230FE96E010E4B
:104720000320EA6EEF50200804E1D6C3D8F3010E4F
:10473000D66FD607EDD7010EEA6E230EE96EF2CFE3
:10474000D9F3F29E000E0001B7EC03F00A00090055
:10475000F550EE6E0009FBE10301D9BFF28E6851FE
:104760000E0826E30E0ED8806855006ED8900032F1
:104770000050230FDA6F010EDB6FD8B0DB2B0B0E6E
:104780006225DC6FDD6BD8B0DD2B040EDC25DE6F1F
:10479000000EDD21DF6FDBC3E1F3DAC3E0F3E36F8B
:1047A000DEC3E2F368C3E4F3000105DE86D0030153
:1047B00068511B08D8A082D00B0E6225D96FDA6B26
:1047C000D8B0DA2B040ED925DB6F000EDA21DC6FAE
:1047D000010EE16F230EE06FDCC3E3F3DBC3E2F312
:1047E00068C3E4F30001E7DD0E0E0301D66FD65176
:1047F000010810E2036AD651230FE96E010E03206F
:10480000EA6EEF50200804E1D6C3D8F3010ED66F4C
:10481000D607EDD7D851685DD76FD7510E0802E2A1
:104820000E0ED76F010EEA6E230EE96EF2CFD9F3AA
:10483000F29E000E0001B7EC03F00A000900F550EB
:10484000EE6E0009FBE10301D9BFF28E0B0E62256B
:10485000D96FDA6BD8B0DA2B040ED925DB6F000ED6
:10486000DA21DC6F010EE16F230EE06FDCC3E3F3AE
:10487000DBC3E2F3D8C3E4F300019DDD0B0E0301BB
:104880006225D96FDA6BD8B0DA2B040ED925DB6F2D
:10489000000EDA21DC6FD851DB25DD6F000EDC2144
:1048A000DE6F010EE16F310EE06FDEC3E3F3DDC3B7
:1048B000E2F3D7C3E4F300017EDD03016251EF08A8
:1048C00014E2010EEA6E230EE96EF2CFD9F3F29EE6
:1048D000000E00011EEC04F00A000900F550EE6E17
:1048E0000009FBE10301D9BFF28E000161EF25F061
:1048F0000C0E0501C76F00014EEC06F0030EEA6EC8
:104900002E0EE96EF2CFD6F3F29E000E5FEC03F0AE
:104910000A000900F550EE6E0009FBE10301D6BF65
:10492000F28E030EEA6E330EE96EF2CFD6F3F29EEC
:10493000000E00016AEC03F00A000900F550EE6E6B
:104940000009FBE10301D6BFF28E030EEA6E380EBA
:10495000E96EF2CFD6F3F29E000E000175EC03F083
:104960000A000900F550EE6E0009FBE10301D6BF15
:10497000F28E030EEA6E3D0EE96EF2CFD6F3F29E92
:10498000000E000180EC03F00A000900F550EE6E05
:104990000009FBE10301D6BFF28E030EEA6E420E60
:1049A000E96EF2CFD6F3F29E000E00018BEC03F01D
:1049B0000A000900F550EE6E0009FBE10301D6BFC5
:1049C000F28E030EEA6E470EE96EF2CFD6F3F29E38
:1049D000000E000196EC03F00A000900F550EE6E9F
:1049E0000009FBE10301D6BFF28E030EEA6E4C0E06
:1049F000E96EF2CFD6F3F29E000E0001A1EC03F0B7
:104A00000A000900F550EE6E0009FBE10301D6BF74
:104A1000F28E030EEA6E510EE96EF2CFD6F3F29EDD
:104A2000000E0001ACEC03F00A000900F550EE6E38
:104A30000009FBE10301D6BFF28EEA6A0B0EE96EB4
:104A4000F2CFD6F3F29E000E000138EC01F00A001E
:104A50000900F550EE6E0009FBE10301D6BFF28EAE
:104A6000010EEA6E060EE96EF2CFD6F3F29E000E4C
:104A70000001B7EC03F00A000900F550EE6E0009E2
:104A8000FBE10301D6BFF28E010EEA6E230EE96E42
:104A9000F2CFD6F3F29E000E0001B7EC03F00A004D
:104AA0000900F550EE6E0009FBE10301D6BFF28E5E
:104AB000D76B0B0ED66F000185EF1FF045EF20F08E
:104AC000B9D4200E9EA8FED7AD6E030E0301D66F9B
:104AD0002A0E9EA8FED7AD6ED62FFAD7200E9EA81E
:104AE000FED7AD6E010EEA6E230EE96E000EEF10DA
:104AF00008E0EF509EA8FED7AD6EE92AD8B4EA2AA6
:104B0000F5D7200E9EA8FED7AD6E2A0E9EA8FED722
:104B1000AD6E200E9EA8FED7AD6E010EEA6E060E9B
:104B2000E96E000EEF1008E0EF509EA8FED7AD6EC4
:104B3000E92AD8B4EA2AF5D7200E9EA8FED7AD6E92
:104B4000030ED86F2A0E9EA8FED7AD6ED82FFAD7C7
:104B5000200E9EA8FED7AD6E030EE16FB80EE06F7B
:104B6000010EE36F230EE26F0E0EE46F000123DCF3
:104B70000301C66B030EE16FC70EE06F010EE36F1A
:104B8000310EE26F0E0EE46F000115DC0301D56BF0
:104B9000030EE16F9A0EE06F010EE36F060EE26FF7
:104BA0000E0EE46F000107DC0301A86B030EE16F3A
:104BB000A90EE06F010EE36F140EE26F0E0EE46FAC
:104BC0000001DBEC21F00301B76B0101CE8F050181
:104BD000C46BC56B000155EC06F0030EEA6EB80E0F
:104BE000E96E000EEF1010E0EACFD7F3E9CFD6F36D
:104BF000EFCFC7F54DEC08F0D7C3EAFFD6C3E9FF06
:104C0000E92AD8B4EA2AEDD70501C46B010EC56FB5
:104C1000000155EC06F0030EEA6EC70EE96E000EB9
:104C2000EF1010E0EACFD7F3E9CFD6F3EFCFC7F517
:104C30004DEC08F0D7C3EAFFD6C3E9FFE92AD8B4A0
:104C4000EA2AEDD70101CE9F0501C46B020EC56FA4
:104C5000000155EC06F0030EEA6E9A0EE96E000EA6
:104C6000EF1010E0EACFD7F3E9CFD6F3EFCFC7F5D7
:104C70004DEC08F0D7C3EAFFD6C3E9FFE92AD8B460
:104C8000EA2AEDD70501C46B030EC56F000155EC90
:104C900006F0030EEA6EA90EE96E000EEF1010E0AA
:104CA000EACFD7F3E9CFD6F3EFCFC7F54DEC08F055
:104CB000D7C3EAFFD6C3E9FFE92AD8B4EA2AEDD779
:104CC0000301716B726B0001C5EF31F00301836B5F
:104CD000826B816B806BC5C1DDF5C4C1DCF5C3C1DE
:104CE000DBF5C2C1DAF5030E0501DF6FA40EDE6F3E
:104CF000000179EC0CF003017B6B7A6B796BACC330
:104D000078F37F6B7E6B7D6BADC37CF3783779373F
:104D10007A377B37783779377A377B37783779370F
:104D20007A377B37783779377A377B3778377937FF
:104D30007A377B37783779377A377B3778377937EF
:104D40007A377B37800E78177BC383F37AC382F37D
:104D500079C381F378C380F37C5180277D5181230F
:104D60007E5182237F5183230A0E8027000E8123E8
:104D7000822383230501A46BA4510001FDEC03F001
:104D80000501A42B006E00509EA8FED7AD6E0A0E42
:104D9000A45DF2E1410EE96E83C3CBF582C3CAF58F
:104DA00081C3C9F580C3C8F50001E8EC13F0200EFB
:104DB0009EA8FED7AD6E0A0E9EA8FED7AD6E0D0E54
:104DC0009EA8FED7AD6E35EF27F00301A46B020E4F
:104DD0008027000E81238223832383530AE1825399
:104DE00008E1815101080EE2FF0A03E18051000849
:104DF00009E2A42B000E805F020E815B000E825B35
:104E0000835BEBD7A4510101C2250501A56F000EFC
:104E10000101C3210501A66F000E0101C421050196
:104E2000A76F000E0101C5210501A86FDD6FA7C5A1
:104E3000DCF5A6C5DBF5A5C5DAF5030EDF6FA50E1B
:104E4000DE6F000179EC0CF00301736BA50E802579
:104E5000E96E030E8121EA6EEFCF73F3733B0F0E01
:104E60007317000136EF27F031D7AFD70301A46BDA
:104E7000A4510001CEEC03F00301A42B006E0050FE
:104E80009EA8FED7AD6E060EA45DF2E173C3C4F515
:104E90001B0E0501C56F000167EC08F0200E9EA8EF
:104EA000FED7AD6E0A0E9EA8FED7AD6E0D0E9EA863
:104EB000FED7AD6E0301976B966B956B946B735138
:104EC000090807E1976B010E966FF40E956F946BCE
:104ED0005AD073510A0807E1976B020E966F710E54
:104EE000956F946B50D073510B0807E1976B020ECE
:104EF000966FEE0E956F946B46D07351070807E1DD
:104F0000976B010E966F770E956F946B3CD0735133
:104F10000C0807E1976B030E966F6B0E956F946B01
:104F200032D073510D0807E1976B030E966FE80EB0
:104F3000956F946B28D073510E0807E1976B040EA0
:104F4000966FE20E956F946B1ED0735308E1976BCA
:104F5000030E966F0D0E956F400E946F14D0735123
:104F6000080808E1976B010E966FB50E956F800EDD
:104F7000946F09D073510F0806E1976B966B030E7F
:104F8000956FE80E946FA46BA4510001DCEC03F064
:104F90000301A42B006E00509EA8FED7AD6E0A0E32
:104FA000A45DF2E1410EE96E97C3CBF596C3CAF555
:104FB00095C3C9F594C3C8F50001E8EC13F0200EC1
:104FC0009EA8FED7AD6E0A0E9EA8FED7AD6E0D0E42
:104FD0009EA8FED7AD6E03019731036E9631026E27
:104FE0009531016E9431006E03320232013200328B
:104FF00003320232013200321F0E031603C0A7F340
:1050000002C0A6F301C0A5F300C0A4F38BC3D7F57B
:105010008AC3D6F589C3D5F588C3D4F503C0DBF5BB
:1050200002C0DAF501C0D9F500C0D8F5000139ECAD
:105030000DF003C093F302C092F301C091F300C0DE
:1050400090F30301A46BA4510001EDEC03F0030104
:10505000A42B006E00509EA8FED7AD6E0A0EA45D74
:10506000F2E1410EE96E93C3CBF592C3CAF591C349
:10507000C9F590C3C8F50001E8EC13F0200E9EA816
:10508000FED7AD6E93C3D7F592C3D6F591C3D5F5D0
:1050900090C3D4F50501DB6BDA6BD96B3C0ED86F8E
:1050A000000139EC0DF000C070F3030170513C0DAC
:1050B000F350905D6F6F360E0501C46F040EC56F1F
:1050C000000155EC06F070C3C5F5110E0501C66F61
:1050D00000014AEC14F03A0E0501C76F00014DECD7
:1050E00008F0480E0501C46F040EC56F000155ECB1
:1050F00006F06FC3C5F5010E0501C66F00014AEC4D
:1051000014F0CBEF31F0EACFB2F3E9CFB1F3030102
:10511000AB39F009AD6FAD27E20FAE6F320FB06F54
:10512000AB510F0BAE27AE27B027E90FAF6FAF27FC
:10513000AF27AA390F0BAF27B027AF37B037B01F53
:10514000B037AA510F0BB027AD37070EAC6F0A0E60
:10515000AF07B027FDE3AE07AF27FDE3AD07AE27EE
:10516000FDE3AC07AD27FDE3030EEA6EAC0EE96E7E
:10517000070EB115B19DE926B00EE95CD8B4B18D2A
:10518000EF50006E08E1B1BD06D0B1B916D0B1B78D
:1051900002D0200E03D0B187B199300E0026EACF9D
:1051A000ABF3E9CFAAF300C0C7F500014DEC08F05E
:1051B000ABC3EAFFAAC3E9FF0301EE50B1ADDCD7F0
:1051C0000001000C7E0E0501C86F000166EC06F0C0
:1051D0007E0E0501C86F000166EC06F00501C86B84
:1051E000000166EC06F00501C86B000166EC06F0F4
:1051F0007E0E0501C86F000166EC06F07E0E05010B
:10520000C86F000166EC06F00501C86B000166EC92
:1052100006F0000C0101CE990201DEB1C0D021C31D
:10522000A3F520C3A2F51FC3A1F51EC3A0F5050178
:10523000AF6B0201F2510501A1259C6F0201F351F0
:105240000501A2219D6F0201F4510501A3219E6F6A
:105250000201F5510501AF219F6F9FC5DDF59EC588
:10526000DCF59DC5DBF59CC5DAF5030EDF6F980E06
:10527000DE6F000179EC0CF00501006A0050A05DC2
:10528000B06FA151A159B16FA251A259B26FA351F0
:10529000A359B36FD890B035A86FB135A96FB235A7
:1052A000AA6FB335AB6FABC59BF5AAC59AF5A9C577
:1052B00099F5A8C598F59B53D8A46ED09A53D8A455
:1052C0006BD099510108D8A067D003E19851FE082E
:1052D00063E3010E9825AC6F000E9921AD6F000EAF
:1052E0009A21000E9B21980EAC25E96E030EAD218C
:1052F000EA6EEF50B26BB16BB06FB56B980E98253C
:10530000E96E030E9921EA6EEF50B525A46F000EE9
:10531000B021A56F000EB121A66F000EB221A76FBC
:10532000A7530AE1A65308E1A551FE0808E2FF0AC7
:1053300003E1A451EF0803E2000E016E95D1010EC6
:10534000A025006E000EA121016E000EA221026EAA
:10535000000EA321036E0050A45D09E10150A55D7C
:1053600006E10250A65D03E10350A75D06E00101DE
:10537000CE89010E016E050177D1A7C5A3F5A6C59B
:10538000A2F5A5C5A1F5A4C5A0F5020E9827000EAB
:1053900099239A239B238FD74BD766D10201DEA195
:1053A00064D121C3A3F520C3A2F51FC3A1F51EC379
:1053B000A0F50501A331AF6FA231AE6FA131AD6F82
:1053C000A031AC6FAF33AE33AD33AC33AF33AE33AC
:1053D000AD33AC33AF33AE33AD33AC33AF33AE33C9
:1053E000AD33AC33AF33AE33AD33AC33AF33AE33B9
:1053F000AD33AC33010EAF170201F2510501AC25FC
:105400009C6F0201F3510501AD219D6F0201F45122
:105410000501AE219E6F0201F5510501AF219F6F7D
:105420009FC5DDF59EC5DCF59DC5DBF59CC5DAF5B0
:10543000030EDF6F980EDE6F000179EC0CF00501B2
:10544000A331AF6FA231AE6FA131AD6FA031AC6FA0
:10545000AF33AE33AD33AC33AF33AE33AD33AC3348
:10546000AF33AE33AD33AC33AF33AE33AD33AC3338
:10547000AF33AE33AD33AC33AF33AE33AD33AC3328
:10548000010EAF17AC35006EAD35016EAE35026E54
:10549000AF35036E0036013602360336003601366C
:1054A0000236033600360136023603360036013640
:1054B0000236033600360136023603360036013630
:1054C00002360336800E00160050A05DB06F01500A
:1054D000A159B16F0250A259B26F0350A359B36FD3
:1054E000B035A86FB135A96FB235AA6FB335AB6FC0
:1054F000A837A937AA37AB37FC0EA817ABC59BF561
:10550000AAC59AF5A9C599F5A8C598F59B53D8A43D
:10551000AAD09A53D8A4A7D099510108D8A0A3D053
:1055200004E19851FC08D8A09ED0030E9825AC6FDA
:10553000000E9921AD6F000E9A21000E9B21980E4E
:10554000AC25E96E030EAD21EA6EEF50B06FB56B7E
:10555000B66BB76B020E9825B96F000E9921BA6F22
:10556000000E9A21000E9B21980EB925E96E030EBC
:10557000BA21EA6EEF50BE6BBD6F006A016A00503F
:10558000B525A46F0150B621A56FBD51B721A66FF7
:10559000BE51B021A76F010E9825AC6F000E992166
:1055A000AD6F000E9A21000E9B21980EAC25E96E7E
:1055B000030EAD21EA6EEF50B26BB16BB06FB56BFD
:1055C000980E9825E96E030E9921EA6EEF50B525E5
:1055D000006E000EB021016E000EB121026E000EB1
:1055E000B221036E0050A4270150A5230250A62328
:1055F0000350A723A43D0AD0A53D08D0A63D06D060
:10560000A7510F0803E1000E016E2ED0010EA02558
:10561000006E000EA121016E000EA221026E000E8E
:10562000A321036E0050A45D09E10150A55D06E1D0
:105630000250A65D03E10350A75D06E00101CE899B
:10564000010E016E050110D0A7C5A3F5A6C5A2F5F0
:10565000A5C5A1F5A4C5A0F5040E9827000E9923B1
:105660009A239B2353D7A6D60201000194EF32F070
:105670000501C86B000166EC06F0FF0E0501C86F5E
:10568000000166EC06F07E0E0501C86F000166ECB5
:1056900006F03C0E0501C86F000166EC06F0180E1E
:1056A0000501C86F000166EC06F00501C86B00013A
:1056B00066EC06F00501C86B000166EC06F0000C14
:1056C0000201DE93DEB118D0D89003012635006EBA
:1056D0002735016E2835026E2935036E00500225EC
:1056E000986F01500321996F025004219A6F035063
:1056F00005219B6F1ED00201DEA11BD003012635C0
:10570000006E2735016E2835026E2935036E00368E
:10571000013602360336FC0E001600500225986F43
:1057200001500321996F025004219A6F0350052103
:105730009B6F0101CEA910D19BC3BAF59AC3B9F5ED
:1057400099C3B8F598C3B7F5000113EC0CF003C08A
:105750009FF302C09EF301C09DF300C09CF3010EB5
:1057600003019825A06F000E9921A16F000E9A21C8
:10577000A26F000E9B21A36FE8CFBAF5A2C3B9F5C3
:10578000A1C3B8F5A0C3B7F5000113EC0CF003C03A
:10579000A4F302C0A3F301C0A2F300C0A1F302C0AE
:1057A00003F001C002F000C001F0006A00500301E4
:1057B0009C252A6F01509D212B6F02509E212C6F3A
:1057C00003509F212D6F0201DEB135D003012C6BF8
:1057D0002D6B2D5328E12C5326E12B51FF0823E399
:1057E00003E12A51EF081FE3D8902A35006E2B35CC
:1057F000016E2C35026E2D35036E00500225986F18
:1058000001500321996F025004219A6F0350052122
:105810009B6F010E0101C627D8B0C72BD8B4C82B87
:10582000D8B4C92B06D00201DE83010E016EC6D0AA
:10583000010192D00201DEA18ED0030E0301982552
:105840009C6F000E99219D6F000E9A219E6F000E95
:105850009B219F6FE8CFBAF59EC3B9F59DC3B8F5FC
:105860009CC3B7F5000113EC0CF003C0A0F302C019
:105870009FF301C09EF300C09DF300C0A5F3030198
:10588000A26BA36BA46B020E9825A66F000E992144
:10589000A76F000E9A21A86F000E9B21A96FE8CF79
:1058A000BAF5A8C3B9F5A7C3B8F5A6C3B7F5000103
:1058B00013EC0CF003C0AAF302C0A9F301C0A8F3D3
:1058C00000C0A7F301C003F000C002F0006A016A43
:1058D0000301A2510026A3510122A4510222A55185
:1058E000032200502A2701502B2302502C2303505F
:1058F0002D232A3D07D02B3D05D02C3D03D02D5123
:105900000F0824E02A35006E2B35016E2C35026E0F
:105910002D35036E0036013602360336FC0E0016B6
:1059200000500225986F01500321996F0250042105
:105930009A6F035005219B6F010E0101C627D8B055
:10594000C72BD8B4C82BD8B4C92B06D00201DE832C
:10595000010E016E33D00101CEB92DD0010E03012D
:1059600026252A6F000E27212B6F000E28212C6F71
:10597000000E29212D6F010E0101C627D8B0C72BBB
:10598000D8B4C82BD8B4C92B03011A510101C65D84
:1059900012E103011B510101C75D0DE103011C511F
:1059A0000101C85D08E103011D510101C95D03E169
:1059B0000201DE830101000E016E02010001000CF4
:1059C0000301A06BA16BA26BA36B0101CEA1BED0A2
:1059D00003017153D8B402D00101B8D00101C651FE
:1059E00003011A5D006E0101C75103011B59016ECD
:1059F0000101C85103011C59026E0101C951030183
:105A00001D59036E00501A5DAA6F01501B59AB6FF0
:105A100002501C59AC6F03501D59AD6FD890AE6B3E
:105A2000AA35AF6FAB35B06FAC35B16FE8CFCAF503
:105A3000B0C3C9F5AFC3C8F5AEC3C7F50501CE6B9A
:105A4000CD6BCC6BE0C2CBF50001FAEC0CF003C0DF
:105A5000A9F302C0A8F301C0A7F300C0A6F3030195
:105A60009731036E9631026E9531016E9431006E5E
:105A7000033202320132003203320232013200328A
:105A80001F0E031603C0ADF302C0ACF301C0ABF3AD
:105A900000C0AAF3A9C3D7F5A8C3D6F5A7C3D5F507
:105AA000A6C3D4F503C0DBF502C0DAF501C0D9F511
:105AB00000C0D8F5000139EC0DF003C093F302C02B
:105AC00092F301C091F300C090F393C3D7F592C352
:105AD000D6F591C3D5F590C3D4F50501DB6BDA6B30
:105AE000D96B3C0ED86F000139EC0DF000C070F39B
:105AF000030170513C0DF350905D6F6F360E050140
:105B0000C46F050EC56F000155EC06F070C3C5F5F6
:105B1000110E0501C66F00014AEC14F03A0E0501A2
:105B2000C76F00014DEC08F0480E0501C46F050E6B
:105B3000C56F000155EC06F06FC3C5F5010E0501F8
:105B4000C66F00014AEC14F079D00101CEA128D033
:105B500003017153D8A402D0010122D0360E0501F1
:105B6000C46F050EC56F000155EC06F0200E05014F
:105B7000C76F00014DEC08F0030E0301AA6F2D0E54
:105B80000501C76F00014DEC08F00301AA2FF7D7FC
:105B9000200E0501C76F00014DEC08F04FD0010148
:105BA000CEB14DD0030E0301AA6F040EAB6FFF0EF2
:105BB000AC6FAD6F000182EC13F00301936B926B3D
:105BC00002C091F301C090F393C3D7F592C3D6F509
:105BD00091C3D5F590C3D4F50501DB6BDA6BD96BB6
:105BE0003C0ED86F000139EC0DF000C070F30301DA
:105BF00070513C0DF350905D6F6F81A201D035D292
:105C0000360E0501C46F050EC56F000155EC06F098
:105C100070C3C5F5110E0501C66F00014AEC14F002
:105C20003A0E0501C76F00014DEC08F06FC3C5F5D2
:105C3000010E0501C66F00014AEC14F0010181A2BA
:105C400002D0030112D20501C46B050EC56F00011D
:105C500055EC06F080B007D0210E0501C76F00019A
:105C60004DEC08F001D004DD030E0301AA6F050E10
:105C7000AB6FFF0EAC6FAD6F000182EC13F002C092
:105C8000A3F301C0A2F30301A251FE0BA46FA3C3AF
:105C9000A5F30501C46B040EC56F000155EC06F0B9
:105CA000000EE96EA5C3ABF3A4C3AAF383EC28F0FE
:105CB00081A202D00301D9D1030E0301AA6F080EFD
:105CC000AB6FFF0EAC6FAD6F000182EC13F002C042
:105CD000A1F301C0A0F30301A1C3A0F3A16BA13301
:105CE000A033A133A033A133A033A133A0330F0ECF
:105CF000A11781A201D0B9D17051090809E2210E82
:105D00000501C46F040EC56F000155EC06F008D004
:105D1000240E0501C46F040EC56F000155EC06F09A
:105D20000301A0510E0816E1A15314E1330E050141
:105D3000C76F00014DEC08F0320E0501C76F00017E
:105D40004DEC08F0300E0501C76F00014DEC08F076
:105D500043D10301A0510D0816E1A15314E1320E05
:105D60000501C76F00014DEC08F0350E0501C76F46
:105D700000014DEC08F0360E0501C76F00014DEC37
:105D800008F02AD10301A0510C0816E1A15314E137
:105D9000320E0501C76F00014DEC08F0320E05010F
:105DA000C76F00014DEC08F0340E0501C76F00010C
:105DB0004DEC08F011D10301A0510B0816E1A153DD
:105DC00014E1310E0501C76F00014DEC08F0390EEA
:105DD0000501C76F00014DEC08F0320E0501C76FD9
:105DE00000014DEC08F0F8D00301A0510A0816E1BB
:105DF000A15314E1310E0501C76F00014DEC08F00D
:105E0000360E0501C76F00014DEC08F0300E05019C
:105E1000C76F00014DEC08F0DFD00301A051090865
:105E200016E1A15314E1310E0501C76F00014DECDD
:105E300008F0320E0501C76F00014DEC08F0380E76
:105E40000501C76F00014DEC08F0C6D00301A05159
:105E5000080816E1A15314E1310E0501C76F0001D6
:105E60004DEC08F0310E0501C76F00014DEC08F054
:105E7000320E0501C76F00014DEC08F0ADD00301F3
:105E8000A051070816E1A15314E1200E0501C76FC8
:105E900000014DEC08F0390E0501C76F00014DEC13
:105EA00008F0360E0501C76F00014DEC08F094D0E4
:105EB0000301A051060816E1A15314E1200E0501CB
:105EC000C76F00014DEC08F0380E0501C76F0001E7
:105ED0004DEC08F0300E0501C76F00014DEC08F0E5
:105EE0007BD00301A051050816E1A15314E1200E57
:105EF0000501C76F00014DEC08F0360E0501C76FB4
:105F000000014DEC08F0340E0501C76F00014DECA7
:105F100008F062D00301A051040816E1A15314E176
:105F2000200E0501C76F00014DEC08F0350E05018C
:105F3000C76F00014DEC08F0360E0501C76F000178
:105F40004DEC08F049D00301A051030816E1A1531C
:105F500014E1200E0501C76F00014DEC08F0340E6E
:105F60000501C76F00014DEC08F0380E0501C76F41
:105F700000014DEC08F030D00301A051020816E1F9
:105F8000A15314E1200E0501C76F00014DEC08F08C
:105F9000340E0501C76F00014DEC08F0300E05010D
:105FA000C76F00014DEC08F017D00301A02D15D0EC
:105FB000A15313E1200E0501C76F00014DEC08F05D
:105FC000330E0501C76F00014DEC08F0320E0501DC
:105FD000C76F00014DEC08F0030181A201D045D04C
:105FE000715327E1725308E1A1C375F3A0C374F3A1
:105FF000A1C377F3A0C376F3722D04D0A1C375F3C8
:10600000A0C374F37251020804E1A1C377F3A0C3E3
:1060100076F381A201D029D0722B72510308D8B433
:10602000726B7651745D03E17751755D02E0010E8C
:10603000716F71531AE0360E0501C46F040EC56FFF
:10604000000155EC06F00301AA6BAA5100012EECE9
:1060500004F00301AA2B006EE8CFC7F500014DEC58
:1060600008F0050E0301AA5DF0E10001000C80922A
:10607000FF0E0501F06F0001AAEC09F09AC3A1F32D
:106080009BC3A2F399C3A4F398C3A3F3510E0501D4
:10609000E86F9BC3EAF59AC3E9F599C3ECF598C399
:1060A000EBF5010EED6F0001F1EC0BF0FF0E0501B9
:1060B000F06F0001AAEC09F001C09FF303019F53A8
:1060C00002E00001F3D7FF0E0501F06F0001AAEC1A
:1060D00009F00150FE0802E00301F5D70201DEB32A
:1060E00030D003019D6B9D5110082AE081B20BD086
:1060F000E1C18FF3E0C18EF3DFC18DF3DEC18CF31C
:1061000000015EDC030181B201D0FDD79C6B9C5184
:10611000200814E081888088070E9E6F9E3D01D084
:106120000AD08094808480A6819680B681868184FE
:1061300081949E07F3D781989C2BE9D79D2BD3D7C9
:106140000201DEA343D003019D6B9D5110083EE088
:1061500081B20BD0E1C18FF3E0C18EF3DFC18DF3CB
:10616000DEC18CF300012CDC030181B201D0FDD72C
:106170009C6B9C51200828E081888088070E9E6FC8
:106180009E3D01D01ED0809480840101CA5308E155
:10619000CB5306E1CC5304E1CD5302E181960CD000
:1061A000FF0ECA27D8A0CB27D8A0CC27D8A0CD27B0
:1061B00080A6819680B681868184819403019E07A2
:1061C000DFD781989C2BD5D79D2BBFD7FF0E05011C
:1061D000F06F0001AAEC09F0FF0E0501F06F00015D
:1061E000AAEC09F08082000E016E10EF35F001017B
:1061F000CEA716D00001D3EF1EF002C0DBF101C024
:10620000DAF10101D751DB5D06E303E1DA51D65D36
:1062100002E2F0D705D0DA5303E1DB5301E1EAD71C
:1062200000010EEC1FF04DEF1FF00101CE91ED6B60
:10623000EC6BEB6BEA6BCE93CEBB08D0010E030187
:10624000986F0001E2EC14F009D00101CEAB07D049
:10625000020E0301986F0001E2EC14F00101D890E6
:10626000E26BC235E36FC335E46FC435E56F0301FC
:10627000986B9851000104EC05F00301982B006E17
:1062800000509EA8FED7AD6E0C0E985DF2E1020E96
:10629000E96EDBC1C4F5DAC1C3F500018DEC14F081
:1062A0002F0E9EA8FED7AD6E100EE96ED7C1C4F5B5
:1062B000D6C1C3F58DEC14F0200E9EA8FED7AD6EAE
:1062C0000101CEA54BD00301986B9851000117EC4A
:1062D00005F00301982B006E00509EA8FED7AD6E0E
:1062E0000A0E985DF2E1410EE96EE5C1CBF5E4C11D
:1062F000CAF5E3C1C9F5E2C1C8F50001E8EC13F045
:10630000200E9EA8FED7AD6E0301986B9851000138
:1063100027EC05F00301982B006E00509EA8FED7D5
:10632000AD6E100E985DF2E1410EE96E25C3CBF51E
:1063300024C3CAF523C3C9F522C3C8F50001E8EC9C
:1063400013F0200E9EA8FED7AD6E0A0E9EA8FED7B3
:10635000AD6E0D0E9EA8FED7AD6E0101C5C187F3CF
:10636000C4C186F3C3C185F3C2C184F325C38BF3D3
:1063700024C38AF323C389F322C388F3DBC199F3CF
:10638000DAC198F3000178EF24F0DBC199F3DAC1A8
:1063900098F334EF27F00C0E0501C46F050EC56F9E
:1063A000000155EC06F0020EE96EDBC1ABF3DAC179
:1063B000AAF383EC28F02F0E0501C76F00014DEC06
:1063C00008F0240E0501C46F050EC56F000155ECE1
:1063D00006F0100EE96ED7C1ABF3D6C1AAF383EC79
:1063E00028F0020E0301AA6F0B0EAB6FDDC1ACF3F8
:1063F000DDC1ADF3000182EC13F003011D6B1C6BDA
:106400001B6B010E1A6F05019D6BE0C29CF5020E1D
:106410009F6F9E6B000128EC0DF002C099F301C044
:1064200098F30501CA6BC96B02C0C8F501C0C7F576
:106430001DC3CEF51CC3CDF51BC3CCF51AC3CBF5DC
:106440000001FAEC0CF003500301255D15E30BE1AC
:106450000250245D11E307E10150235D0DE303E1E8
:106460002251005C09E2010E1A27D8B01B2BD8B4C8
:106470001C2BD8B41D2BC7D7010E1A5D986F000EC8
:106480001B59996F000E1C599A6F000E1D599B6F76
:10649000E8CFCAF59AC3C9F599C3C8F598C3C7F53B
:1064A0000501CE6BCD6BCC6BE0C2CBF50001FAECF5
:1064B0000CF003C09CF302C09BF301C09AF300C030
:1064C00099F3D890006A03019935016E9A35026EEE
:1064D0009B35036E0050225D0101CA6F015003011C
:1064E00023590101CB6F0250030124590101CC6FE4
:1064F0000350030125590101CD6FC96BC86BC76BF0
:10650000C66B21C329F320C328F31FC327F31EC37F
:1065100026F30501C46B050EC56F000155EC06F0AE
:10652000E2EC28F00AEF29F00101CEA510D003011A
:10653000986B985100013BEC05F00301982B006E1D
:1065400000509EA8FED7AD6E110E985DF2E10501D8
:10655000C46B050EC56F000155EC06F038EC2BF04E
:106560000101C95103011D5DD8A074D214E10101DC
:10657000C85103011C5DD8A06DD20DE10101C751C6
:1065800003011B5DD8A066D206E10101C6510301DB
:106590001A5DD8A05FD2000160EC2BF0020E03015F
:1065A000265D986F000E2759996F000E28599A6F33
:1065B000000E29599B6FE8CFCAF59AC3C9F599C354
:1065C000C8F598C3C7F50501CE6BCD6BCC6BE0C2A7
:1065D000CBF50001FAEC0CF003C0F1F102C0F0F1D0
:1065E00001C0EFF100C0EEF1030112510101EE27ED
:1065F000030113510101EF23030114510101F023A1
:10660000030115510101F1230201DEA108D0E0517F
:106610000101EE5F000EEF5BF05BF15B0201D890D1
:106620000101E66BEE35E76FEF35E86FF035E96FA6
:106630008092FF0E0501F06F0001AAEC09F0500EE8
:106640000501E36FE56BE46B020EE76FE66BFF0E8F
:10665000E86F0001D4EC09F0015202E00101E9D732
:10666000FF0E0501F06F0001AAEC09F0FF0E050115
:10667000F06F0001AAEC09F08082E9C1E1F1E8C104
:10668000E0F1E7C1DFF1E6C1DEF1030106510101EE
:10669000E625006E030107510101E721016E0301A8
:1066A00008510101E821026E030109510101E921AC
:1066B000036E0050DE5D0AE10150DF5D07E102502C
:1066C000E05D04E10350E15DD8B4B2D184A00FD005
:1066D000DA2BD8B4DB2BD751DB5D07E303E1DA51CA
:1066E000D65D03E2DB6B010EDA6F82D552D080AA51
:1066F0000DD0DA51D8B4DB07DA2F06D0DB5304E132
:10670000D7C1DBF1D6C1DAF173D543D084A420D050
:10671000DD5110081DE20501C46B050EC56F0001B7
:1067200055EC06F02B0E0501C76F00014DEC08F08B
:106730000101DD07020E0301AA6F0B0EAB6FDDC175
:10674000ACF3DDC1ADF3000182EC13F021D0010107
:1067500084A21FD0DD3D01D01CD00501C46B050E05
:10676000C56F000155EC06F02D0E0501C76F000145
:106770004DEC08F00101DD2B020E0301AA6F0B0E98
:10678000AB6FDDC1ACF3DDC1ADF3000182EC13F002
:106790000101ED6BEC6BEB6BEA6B83AE41D0010E4C
:1067A000EA27D8B0EB2BD8B4EC2BD8B4ED2B010EE4
:1067B00003019E6F000127EC06F00101CEB32FD03C
:1067C000ED5307E1EC5305E1EB5303E1EA51F9081E
:1067D00026E20501C46B050EC56F000155EC06F0FD
:1067E0003E0E0501C76F00014DEC08F00101CE819E
:1067F000CE930201DEB312D0000160EC2BF0020157
:10680000DEB30CD02DC329F32CC328F32BC327F3FD
:106810002AC326F30001E0EC2CF002010101BDD7F0
:10682000CEB324D0EA5306E1EB5304E1EC5302E18A
:10683000ED531CE0ED531AE1EC5318E1EB5316E174
:10684000EA51F90813E3CE830501C46B050EC56F49
:10685000000155EC06F0E2EC28F0140E03019E6FE7
:10686000000127EC06F0010194D7CFD0CEA31AD0B7
:10687000EA5306E1EB5304E1EC5302E1ED5312E07D
:10688000CE930501C46B050EC56F000155EC06F0F3
:1068900038EC2BF0140E03019E6F000127EC06F07C
:1068A000B5D00101CEA3B1D0CEAD2AD0DC6B0001B2
:1068B0000EEC1FF00501C46B050EC56F000155EC11
:1068C00006F00101CE8F0301986B985100014CEC4A
:1068D00005F00301982B006EE8CFC7F500014DECE1
:1068E00008F00E0E0301985DF0E10101CE9F030E4A
:1068F0000301986F0001E2EC14F00101CE8BCE9DF4
:1069000084A234D0CE8BD551D35DD8A0D32B060E24
:106910000301986F2A0E9EA8FED7AD6E982FFAD766
:10692000996B995100015CEC05F00301992B006E05
:1069300000509EA8FED7AD6E0D0E995DF2E1D3C159
:10694000C4F51B0E0501C56F000167EC08F0200EB1
:106950009EA8FED7AD6E0A0E9EA8FED7AD6E0D0E98
:106960009EA8FED7AD6E0101CE8D35D084A433D064
:10697000CE8BD3510008D8A0D307060E0301986F21
:106980002A0E9EA8FED7AD6E982FFAD7996B995113
:1069900000015CEC05F00301992B006E00509EA8ED
:1069A000FED7AD6E0D0E995DF2E1D3C1C4F51B0E9D
:1069B0000501C56F000167EC08F0200E9EA8FED708
:1069C000AD6E0A0E9EA8FED7AD6E0D0E9EA8FED728
:1069D000AD6E0101CE8D83AE11D0CEAB0FD0020EC5
:1069E0000301AA6F0B0EAB6FFF0EAC6FAD6F000112
:1069F00082EC13F0F7EF30F009D0010183AE04D040
:106A0000CEBB02D0C6D601D04FD70001E1C19BF367
:106A1000E0C19AF3DFC199F3DEC198F337EF30F0AC
:106A2000020E0101DF27000EE023E12300012DD635
:106A30000201DEB309D02DC329F32CC328F32BC3E5
:106A400027F32AC326F303D0DEA301D004D000012C
:106A500087D503010201000180EF38F0F86AD09E6B
:106A6000FE0E006E060E016E020EE96E000EEA6E5C
:106A7000EE6A002EFDD7012EFBD7EA6AE96A0A0EFC
:106A8000AF6EA60EAC6E900EAB6EC180C182C1849B
:106A9000C196056A066A1E0E0101F26F210EF36FA0
:106AA000610EF46F210EF56F120EF66F3C0EF76F4C
:106AB000410EF86F400EF96F210EFA6F7C0EFB6FDE
:106AC000380EFC6F540EFD6F560EFE6F550EFF6FA5
:106AD000180E0201006F200E016F550E026F036F3A
:106AE000046F780E056F200E066F550E076F540E5B
:106AF000086F550E096F780E0A6F200E0B6F550E3A
:106B00000C6F560E0D6F540E0E6F780E0F6F200E19
:106B1000106F540E116F550E126F540E136F780EC6
:106B2000146F1C0E156F220E166F620E176F220E59
:106B3000186F100E196F380E1A6F550E1B6F1C6FE1
:106B40001D6F180E1E6F380E1F6F550E206F540EDE
:106B5000216F550E226F180E236F380E246F540EBE
:106B6000256F550E266F560E276F180E286F296B4E
:106B7000450E2A6F7C0E2B6F410E2C6F2D6B2E6BEA
:106B8000450E2F6F7D0E306F410E316F326B336BC0
:106B9000450E346F7E0E356F400E366F376B780EB4
:106BA000386F150E396F140E3A6F150E3B6F780E55
:106BB0003C6F3D6F140E3E6F150E3F6F140E406F0D
:106BC000780E416F7C0E426F540E436F560E446F29
:106BD000550E456F440E466F240E476F540E486F96
:106BE000780E496F540E4A6F480E4B6F7E0E4C6FF5
:106BF000090E4D6F7E0E4E6F490E4F6F506F380E5F
:106C0000516F450E526F536F546F380E556F566F5C
:106C1000450E576F440E586F450E596F380E5A6F18
:106C20005B6F450E5C6F460E5D6F440E5E6F380EF7
:106C30005F6F3C0E606F410E616F626F210E636F7C
:106C40007C0E646F3C0E656F410E666F420E676F7F
:106C5000200E686F7C0E696F0C0E6A6F510E6B6FA1
:106C6000500E6C6F510E6D6F3C0E6E6F380E6F6F65
:106C7000450E706F440E716F450E726F380E736F54
:106C80003C0E746F410E756F400E766F410E776F3C
:106C90003C0E786F796B7A6B7B6B7C6B7D6B200E17
:106CA0007E6F480E7F6F3E0E806F490E816F620EC1
:106CB000826F836B846B856B866B876B886B896B4C
:106CC0008A6B8B6B8C6B400E8D6F680E8E6F3E0ED9
:106CD0008F6F090E906F020E916F200E926F540EFF
:106CE000936F560E946F550E956F780E966F976B47
:106CF000440E986F7E0E996F410E9A6F9B6B380E03
:106D00009C6F440E9D6F460E9E6F450E9F6F380E12
:106D1000A06F3C0EA16F400EA26F420EA36F210E1A
:106D2000A46F7C0EA56FA66F090EA76F050EA86F46
:106D3000A96F780EAA6F7C0EAB6F090EAC6F110EA7
:106D4000AD6F210EAE6F7C0EAF6F7E0EB06F250E55
:106D5000B16FB26F260EB36F180EB46FC290C180C0
:106D6000C182C184C196290E926E8082020E936EFA
:106D7000900E946EC00E956E968096829684030156
:106D8000986B9851000139EC04F00301982B006EC8
:106D900000509EA8FED7AD6E260E985DF2E1000170
:106DA0006EEF05F0FEEF05F088EC06F0A6EF08F0B8
:106DB0000501C46BC56B000155EC06F00101CE8FD7
:106DC0000301986B9851000155EC04F00301982BD6
:106DD000006EE8CFC7F500014DEC08F00E0E030180
:106DE000985DF0E10101CE9F090E0501C46F010E0F
:106DF000C56F000155EC06F00301986B9851000136
:106E000065EC04F00301982B006EE8CFC7F5000194
:106E10004DEC08F00B0E0301985DF0E10501C46B29
:106E2000020EC56F000155EC06F00301986B9851F6
:106E3000000173EC04F00301982B006EE8CFC7F556
:106E400000014DEC08F00E0E0301985DF0E1030E19
:106E50000501C36F000185EC09F00501C46B040E48
:106E6000C56F000155EC06F00101CEA515D0CE8FFF
:106E70000301986B9851000183EC04F00301982BF7
:106E8000006EE8CFC7F500014DEC08F0050E0301D8
:106E9000985DF0E10101CE9F2A0E0501C46F040E3A
:106EA000C56F000155EC06F00101CEA715D0CE8FBD
:106EB0000301986B985100018EEC04F00301982BAC
:106EC000006EE8CFC7F500014DEC08F0070E030196
:106ED000985DF0E10101CE9F050E0501C36F000131
:106EE00085EC09F0AAEF0AF00101CEA510D003014C
:106EF000986B985100019AEC04F00301982B006EF6
:106F000000509EA8FED7AD6E130E985DF2E1000111
:106F100079EF0DF00101CEA510D00301986B9851C7
:106F20000001ACEC04F00301982B006E00509EA809
:106F3000FED7AD6E180E985DF2E10001AEEF13F0D2
:106F40000101CEA511D00301986B98510001C1EC4D
:106F500004F00301982B006E00509EA8FED7AD6E82
:106F60000F0E985DF2E10101D76BD66BDB6B010E62
:106F7000DA6FD16BD36BD56B0301986B0001E2EC38
:106F800014F00101CEA526D00301986B98510001A1
:106F9000D1EC04F00301982B006E00509EA8FED7A0
:106FA000AD6E0D0E985DF2E1100EE96ED7C1C4F51D
:106FB000D6C1C3F500018DEC14F0200E9EA8FED7BB
:106FC000AD6E0A0E9EA8FED7AD6E0D0E9EA8FED722
:106FD000AD6E0101D650D7CF03F00301986FD7CF24
:106FE00099F39D6B9C6BD7CF9BF39A6F0001A5EF34
:106FF0001EF0200E9EA8FED7AD6E0A0E9EA8FED7EC
:10700000AD6E0D0E9EA8FED7AD6E0101D26BD251B2
:10701000CF5D41E30301986B98510001E3EC04F06C
:107020000301982B006E00509EA8FED7AD6E0B0E8C
:10703000985DF2E1D2C1C4F51B0E0501C56F0001D8
:1070400067EC08F03D0E9EA8FED7AD6E200E9EA800
:10705000FED7AD6E036A0101D251900FE96E010EA9
:107060000320EA6EEFCF98F398C3C4F51B0E050119
:10707000C56F000167EC08F0200E9EA8FED7AD6E2C
:107080000A0E9EA8FED7AD6E0D0E9EA8FED7AD6E61
:107090000101D22BBCD70301986B98510001F3EC8E
:1070A00004F00301982B006E00509EA8FED7AD6E31
:1070B0000B0E985DF2E1D5C1C4F51B0E0501C56F3D
:1070C000000167EC08F0200E9EA8FED7AD6E0A0EF8
:1070D0009EA8FED7AD6E0D0E9EA8FED7AD6E280EF3
:1070E0000101DD6F020E0301AA6F0B0EAB6FDDC154
:1070F000ACF3DDC1ADF3000182EC13F0F7EF30F03B
:107100000101DA2BD8B4DB2BD751DB5D07E303E1B8
:10711000DA51D65D03E2DB6B010EDA6F0001EED7C8
:0271200003006A
:020000040030CA
:0E00000000220C0E000180000FC00FE00F4028
:00000001FF
